:100000000C941E030C9471030C9471030C947103F3
:100010000C9471030C9471030C9471030C94710390
:100020000C9471030C9471030C9495230C9471033C
:100030000C944C310C9471030C9471030C94710367
:100040000C9471030C9471030C9471030C94710360
:100050000C9471030C94D70D0C9471030C947103E0
:100060000C9471030C9471030C9471030C94710340
:100070000C9471030C9471030C9471030C94710330
:100080000C9471030C9471030C9471030C94710320
:100090000C9471030C9471030C9471030C94710310
:1000A0000C9471030C9471030C947103E3210A22E4
:1000B00002230A220223562279220223D022DF229F
:1000C000E627E6271E281E28792A792A792A792AFE
:1000D0009928792A75287528332A792A482A662A80
:1000E000000000000405060708090A0B0C0D0E0F9E
:1000F000101112131415161718191A1B1C1D1E1F88
:10010000202122232425262728292A2B2C2D2E2F77
:10011000303132333435363738393A3B3C3D3E3F67
:10012000404142434445464748494A4B4C4D4E4F57
:10013000505152535455565758595A5B5C5D5E5F47
:10014000606162636465A56768696A6B6C6D6E6FF8
:10015000707172737475767778797A7B7C7D7EA8FE
:10016000A9AA00000085008788898A8B000000000A
:10017000909100000000000000000000000000005E
:10018000000000000000000000000000000000006F
:10019000000000000000000000000000000000005F
:1001A000000000000000000000000000000000004F
:1001B000000000000000000000000000000000003F
:1001C000E0E1E2E3E4E5E6E7000000000000000013
:1001D000000000000000000000000000000000001F
:1001E00073706565643A2025730A007573625F73E6
:1001F000746174653A20253032580A00686F737450
:100200002E5461736B3A2025640A000D0A00200009
:100210000D0A0028686964626F6F742E682920498E
:100220006E746572666163653A000D0A002868693C
:1002300064626F6F742E682920537472616E6765F3
:10024000207265616420636F756E743A20000D0A38
:100250000028686964626F6F742E682920506F6C83
:100260006C3A000D0A0028686964626F6F742E682A
:1002700029206570496E666F5B6570496E746572A2
:1002800072757074496E496E646578202B20695DC3
:100290002E6D6178506B7453697A653D000D0A00CC
:1002A00028686964626F6F742E6829206570496ED2
:1002B000666F5B6570496E74657272757074496EB5
:1002C000496E646578202B20695D2E6570416464F9
:1002D000723D000D0A0028686964626F6F742E68B1
:1002E0002920693D0053657450726F746F3A004263
:1002F0004D20636F6E666967757265640D0A000D47
:100300000A0052504950452072636F64653A000DEF
:100310000A005345545F49444C452072636F64653D
:100320003A000D0A0050524F544F434F4C20534552
:1003300054204849445F424F4F542072636F6465B4
:100340003A000D0A000D0A496E74657266616365B4
:100350003A000D0A00624E756D49666163653A00A8
:100360000D0A006249666163654E756D3A000D0ABB
:1003700000436E663A000D0A00624E756D45503AB4
:10038000004849445F50524F544F434F4C5F4B45D8
:1003900059424F4152440D0A000D0A004E433A00A3
:1003A0000D0A00416464723A000D0A0073657441DD
:1003B0006464723A006570696E666F0D0A00424DA2
:1003C00020496E69740D0A00526F6C6C6F7665720D
:1003D000206572726F723A2069676E6F7265640D84
:1003E0000A000D0A00202530325800696E707574BD
:1003F0002025643A0054332000543220000D0A00B6
:10040000285553423A3A496E5472616E736665726A
:1004100029206570207265717565737465642000AC
:100420000D0A00285553423A3A496E5472616E7370
:1004300066657229206164647220726571756573E6
:1004400074656420000D0A00285553423A3A496EFB
:100450005472616E736665722920536574416464D9
:1004600072657373204661696C65642000436F2078
:100470000054312000436920002E2E2E4641494C65
:100480000D0A0042756666657220706F696E74654C
:1004900072206973204E554C4C210D0A000D0A0044
:1004A0000D0A736574436F6E6620000D0A676574EC
:1004B000446576446573637220000A4B6579626F08
:1004C0006172642073746172742E0A000A5553427B
:1004D00020636F6E666967757265642E0A000A0A8A
:1004E000544D4B3A30323636346665372F4C5546CC
:1004F000410A0A003C0355005300420020007400EA
:100500006F00200055005300420020006B00650082
:10051000790062006F0061007200640020006300D7
:100520006F006E0076006500720074006500720056
:1005300000000E0374002E006D002E006B002E00D4
:1005400000000403090409024200020100A032096C
:1005500004000001030101000921110100012240F2
:10056000000705810308000A0904010002030000D6
:100570000009211101000122220007058203200049
:10058000010705020320000112011001000000080C
:10059000EDFE5B001408010200010631FF0974A1A1
:1005A000010975150026FF0095207508810209765E
:1005B000150026FF00952075089102C00501090667
:1005C000A101050719E029E7150025019508750126
:1005D0008102950175088101050819012905950514
:1005E000750191029501750391010507190029FF15
:1005F000150026FF00950675088100C0636F6E73B5
:10060000756D65723A20253034580A007379737419
:10061000656D3A20253034580A000A0025303258DA
:1006200020006B6579626F6172643A20004C45442A
:100630003A20253032580A00870C420D11241FBE83
:10064000CFEFDAE0DEBFCDBF04B603FE28C0809155
:10065000B5059091B605A091B705B091B805873062
:10066000904BA740B04BD9F41092B5051092B60547
:100670001092B7051092B80514BE0FB6F894A8955D
:1006800080916000886180936000109260000FBECE
:100690001092010810920008E0E0F8E3099511E0DB
:1006A000A0E0B1E0EAEBF7E602C005900D92A638B3
:1006B000B107D9F725E0A6E8B1E001C01D92A53B3E
:1006C000B207E1F713E0CEE1D3E004C02197FE01C9
:1006D0000E94D533CC31D107C9F70E94F51E0C9486
:1006E000DB330C940000FF93EF93E0918601F091CF
:1006F0008701309709F00995EF91FF910895FC016A
:100700008591803011F0EFDFFBCF0895FF27E0E205
:1007100030E247FF0CC0419597FF09C0EDE26095BC
:10072000709580959095611D711D811D911D27FF0C
:1007300002C0219530E350E2AA27660F771F881F79
:10074000991FAA1FA41710F0A41B63955A95A9F727
:10075000AA3008F0A95FA05DAF93F395611571050C
:100760008105910541F7ED3211F4EF93F395F217FE
:1007700018F43F93F395FBCF8F91B5DFFA95E1F72E
:100780000895E991F9918591803021F0853219F031
:10079000AADFF9CF089520E0E89455915532C1F3CE
:1007A000503311F4689455915A3348F4505390F3F0
:1007B000220F022E220F220F200D250FF4CF0EF450
:1007C000219589919991533619F3533729F153356E
:1007D00059F1BC0188279927E8945C3621F4899166
:1007E000999168945591543639F446EF7EF077FF2D
:1007F0000DC08FEF9FEF0AC055374AE039F05835EA
:1008000040E121F0523642E009F00895FF93EF9362
:100810007DDFEF91FF91B7CFFF93EF93FC018191C3
:100820008030B9F360DFFBCFFF93EF9368DFF1CF48
:10083000DF93CF93CDB7DEB72596A3DFCF91DF91BE
:10084000089580E00895089580E0089581E0089576
:10085000CF93DF93CDB7DEB728970FB6F894DEBFFE
:100860000FBECDBFE22F29833A834B835C836D8318
:100870007E838F8398878091C402E82BE093C40223
:10088000FE013396AE01475F5F4F2191243088F01F
:10089000A6ECB2E080E090E03D91311106C0DC01B1
:1008A000AC53BD4F12962C9304C00196863091052F
:1008B00099F7E417F50749F728960FB6F894DEBFC5
:1008C0000FBECDBFDF91CF910895860F911D860F8A
:1008D000911DFC015687458781E00895FC018789B9
:1008E0000895CF93DF93EC018C819D81DC01ED9124
:1008F000FC910480F581E02D6E8109951F86188A90
:1009000081E08A8B1E821B8A1C8A1D8A1E8A1F8A8E
:1009100080E0DF91CF910895FC018681089581E008
:10092000633009F080E0089581E0613009F080E0F3
:100930000895860F911D860F911DFC018585968572
:100940000895EF92FF92CF93DF93DC01E701529677
:100950008C915297823049F11F966C931F97509655
:100960004C9350979B8193709330F9F49A8197FF41
:100970001CC09E8158962C915897291718F45896A8
:100980009C935897E82FF0E09F01220F331FE20F4E
:10099000F31FEA0FFB1F9A819F7097839C819087BA
:1009A00094E091878F5F52968C93DF91CF91FF9067
:1009B000EF900895EF92FF920F9302970E94A10487
:1009C0000F91FF90EF90089508953F924F925F929C
:1009D0006F927F928F929F92AF92BF92CF92DF924F
:1009E000EF92FF920F931F93CF93DF9300D000D02D
:1009F000CDB7DEB76C017C836B835A8349834C018E
:100A000080E1880E911C5601A7E0AA0EB11C11E0EE
:100A100084E0482E3601B2E16B0E711C93E0392E52
:100A200022E0522E8B819C81892B09F4FBC0F601B8
:100A300080A1823059F128F4882341F0813071F08F
:100A4000F1CF833039F18430C1F1ECCF548285810C
:100A50009681908787835286518610A3AE014D5FA1
:100A60005F4FBE016F5F7F4FC5010E94371C882317
:100A700009F4D8C0D6011596ED91FC9116978081A6
:100A800091968C939197818192968C93F6017682C0
:100A9000658230A2D60192968C919297843011F49F
:100AA00093961C92F60181A1825084832581368120
:100AB000308727838287818740A2D60192968C91C6
:100AC0008430B1F0853009F442C0823009F06EC044
:100AD000AE014D5F5F4FBE016F5F7F4FC5010E944A
:100AE000371C882309F49EC0F601858984A392C02F
:100AF000AE014D5F5F4FBE016F5F7F4FC5010E942A
:100B0000371C882309F48EC0D60155968C915597D1
:100B1000833009F07FC056968C915697813009F04A
:100B200079C098969C91989757968C91992321F02B
:100B3000882309F46FC003C0813009F06BC0F6014F
:100B400013A3928996A3938997A385A363C0AE014B
:100B50004D5F5F4FBE016F5F7F4FC5010E94371C25
:100B6000882309F45FC0D60193968C9193978823CC
:100B700009F450C012968D919C911397009709F437
:100B800049C0DC01ED91FC910190F081E02D7401F0
:100B9000D60195960C91959797962C919797969646
:100BA0004C91969794966C91099534C0F601858581
:100BB000882319F0813039F028C081A190E0029794
:100BC0009787868715872B813C8189819A81782F29
:100BD000692FF601468557854115510581F001962B
:100BE0002115310529F41C821B8279836A830DC08B
:100BF000415051095787468721503109E8CF3C833E
:100C00002B839A838983F6011586F601868597855D
:100C1000892B41F4D60116969C928E921597909648
:100C20001C9200CF0F900F900F900F90DF91CF91FB
:100C30001F910F91FF90EF90DF90CF90BF90AF90FA
:100C40009F908F907F906F905F904F903F9008950E
:100C5000CF93DF936091E2017091E301E0918F0106
:100C6000F09190014091D6015091D7012091CA0195
:100C70003091CB018091BE019091BF016E177F072B
:100C8000B1F4E0918D01F0918E014E175F0779F478
:100C9000E0918B01F0918C012E173F0741F4E09118
:100CA0008901F0918A018E179F0709F463C0709340
:100CB000900160938F0150938E0140938D0130938A
:100CC0008C0120938B0190938A0180938901E4EC3D
:100CD000F2E088E0DF011D928A95E9F72091DA01C0
:100CE0003091DB014091DC015091DD016091DE012A
:100CF0007091DF018091E0019091E1010E94280450
:100D00002091CE013091CF014091D0015091D1017D
:100D10006091D2017091D3018091D4019091D5015D
:100D20000E9428042091C2013091C3014091C40166
:100D30005091C5016091C6017091C7018091C801B1
:100D40009091C9010E9428042091B6013091B70109
:100D50004091B8015091B9016091BA017091BB0105
:100D60008091BC019091BD010E94280481E0809394
:100D7000C30202C01092C3020E94B00DEC018CE4C9
:100D800092E00E948316CE010E94C80D853691051F
:100D900060F09F938F938CEF91E09F938F930E94CD
:100DA00018040F900F900F900F908CE492E00E9427
:100DB000080F90918801891779F18CE492E00E94E4
:100DC000080F809388011F928F938BEE91E09F9381
:100DD0008F930E9418040F900F900F900F908091A6
:100DE00088018039C9F480919101823019F08AE13B
:100DF00091E002C085E191E09F938F9380EE91E0B6
:100E00009F938F930E9418040E9483240E94EF25D1
:100E10000F900F900F900F9081E0DF91CF91089588
:100E2000482F80E1489F90011124205E310928302D
:100E3000310538F49091C402992319F0892F90E07C
:100E400002C080E090E0E6ECF2E061E070E0219129
:100E5000243070F0322F32953F70431309C02F7049
:100E6000DB0102C0AA0FBB1F2A95E2F78A2B9B2B3E
:100E7000B2E0EC3CFB0759F708950895CF92DF925A
:100E8000EF92FF920F93CF93DF931F92CDB7DEB710
:100E9000898380914902882371F0CE0101966C010B
:100EA000EE24E394F12C00E022E040E060E082E3F5
:100EB00092E00E94D71780912F02882371F0CE0113
:100EC00001966C01EE24E394F12C00E022E040E076
:100ED00060E088E192E00E94D71780911502882394
:100EE00071F0CE0101966C01EE24E394F12C00E048
:100EF00022E040E060E08EEF91E00E94D717809101
:100F0000FB01882371F0CE0101966C01EE24E3947D
:100F1000F12C00E022E040E060E084EE91E00E94ED
:100F2000D7170F90DF91CF910F91FF90EF90DF9047
:100F3000CF9008950E940A318091AA05882331F04C
:100F40000E943331882321F00C9411200C94280640
:100F50000895FC01758364838EE291E09183808320
:100F60008CE491E093838283138A148A158A168A0B
:100F7000178A418F178288E080878CE381871286E9
:100F8000138684E0848781E0828B118A1786168617
:100F9000158661157105B1F0DB01AA5ABF4F80E0DB
:100FA00090E02D913D91232B49F48B96880F991F4A
:100FB000DB01A80FB91FED93FC93089501968031D2
:100FC000910579F708952E9A08952E988EBD0DB447
:100FD00007FEFDCF1EBC0DB407FEFDCF0E94E30748
:100FE0008EB508952E9882608EBD0DB407FEFDCF9C
:100FF0006EBD0DB407FEFDCF0C94E30788EF0E9491
:10100000E507807C803411F118F4882371F108958C
:10101000803819F0803C39F1089588ED0E94E50789
:101020009091910181FD08C0923029F161EC88ED29
:101030000E94F20782E007C09330E9F063EC88ED8C
:101040000E94F20783E080939101089588ED0E9449
:10105000E5079091910181FD03C0933079F70895E0
:10106000923021F7089581E0EECF61ED88ED0E9486
:10107000F2071092910108950F931F93CF93DF937E
:101080008C01269A0E94E307219A229A2398209A9B
:1010900080E58CBD81E08DBD259868E188E80E94DF
:1010A000F20760E288E70E94F20760E088E70E94AA
:1010B000F207C0E0D0E088E60E94E507219680FDB7
:1010C00006C0CF3F8FEFD807B1F78FEF1DC061EC9F
:1010D00088ED0E94F20760E280ED0E94F20764E072
:1010E00088EE0E94F20788EE0E94E50782FFFBCFA0
:1010F000C8010E94FE0760E288EC0E94F20761E0EE
:1011000080E80E94F20780E0DF91CF911F910F915C
:1011100008958091A60581608093A6058CE492E0F5
:101120000E943C0888ED91E09093400280933F023A
:101130008CEC91E0909326028093250280EC91E064
:1011400090930C0280930B0284EB91E09093F20158
:101150008093F10108950F931F93CF93C82F8B01B4
:10116000282F30E084E0359527958A95E1F780E3D4
:10117000820F8A3310F087E3820FB8010E94721C3D
:10118000CF7080E38C0F8A3310F087E38C0FB801A7
:10119000CF911F910F910C94721C2F923F924F92FE
:1011A0005F926F927F928F929F92AF92BF92CF92F7
:1011B000DF92EF92FF920F931F93CF93DF93CDB700
:1011C000DEB7EB970FB6F894DEBF0FBECDBF7C0144
:1011D000362E242E422EDC011496AD90BC9015972D
:1011E00060E870E08EEB93E00E947F1CF701568070
:1011F000511006C2108ED501ED91FC910190F08145
:10120000E02D60E0C50109956C01009719F446EDE9
:10121000542EFBC1FC01808091808114910449F41B
:1012200060E870E085EB93E00E947F1C37ED532E61
:10123000ECC13701F7E06F0E711CDC0111967C9256
:101240006E9214964C928E01065D1F4F28E030E09E
:1012500040E060E0F701848195810E94D013182F4F
:101260008111B7C11AA5D6018D929C92D501ED913D
:10127000FC910280F381E02D222D40E0632DC50119
:101280000995F7018683882309F4BDC199A9908740
:10129000282F40E060E0848195810E947B14982E85
:1012A000882319F1D60114961C92D501ED91FC9179
:1012B0000480F581E02DD70116966C91C501099542
:1012C000F701168260E870E08CEA93E00E947F1CD0
:1012D00060E870E0892D0E94AB0860E870E089EA60
:1012E00093E00E947F1C592C90C160E870E083EA73
:1012F00093E00E947F1C60E870E0D70116968C9105
:101300000E94AB0860E870E080EA93E00E947F1CD6
:10131000F6011482D501ED91FC910190F081E02D50
:10132000D70116966C91C5010995009709F46FCF06
:10133000212F133108F022E1FC014482211126C043
:101340003BAC60E870E08CE993E00E947F1C60E8B1
:1013500070E0832D0E94AB0860E870E089E993E0BB
:101360000E947F1C60E870E081E893E00E947F1C8F
:10137000412C22E2822E21E0922E5701F2E0AF0EA4
:10138000B11C6E0181E1C80ED11C38C030E08E0165
:10139000065D1F4F40E0D70116966C911697149684
:1013A0008D919C9115970E94D013182F811114C113
:1013B000C7CF9A828982BC82AB821D821A861B8625
:1013C0001E86188A1F8619A21AA21BA219A6DF82DE
:1013D000CE82D986C886DD86CC868E010F5F1F4FF0
:1013E000242D40E0F7016681848195810E941E14BE
:1013F000D70152968C91823019F043944310D9CF83
:1014000060E870E089E793E00E947F1C60E870E08C
:10141000F70182890E94AB0860E870E086E793E0FC
:101420000E947F1CD70152968C915297823009F00E
:10143000D9C0930142E016966C91169714968D913F
:101440009C9115970E94280F60E870E081E793E077
:101450000E947F1C60E870E0F70187850E94AB085E
:1014600060E870E08EE693E00E947F1C68EE73E017
:1014700080E090E00E94590DD7011F962C911F9794
:1014800040E016966C91169714968D919C91159745
:101490000E94E915182F8111A2C068EE73E080E068
:1014A00090E00E94590D60E870E083E693E00E94AE
:1014B0007F1C60E870E0F70180890E94AB0860E85B
:1014C00070E080E693E00E947F1C60E870E085E5B4
:1014D00093E00E947F1C60E870E0D70151968C91E8
:1014E0000E94AB0860E870E082E593E00E947F1CF8
:1014F00060E870E085E493E00E947F1C60E870E0A3
:1015000080E00E94AB0860E870E082E493E00E9413
:101510007F1CF701418D60E0C7010E942E18182F33
:1015200060E870E0811150C085E293E00E947F1C6A
:1015300060E870E080E00E94AB0860E870E082E262
:1015400093E00E947F1C20E040E060E0C7010E9421
:101550000418182F60E870E082E193E00E947F1C7D
:1015600060E870E0812F0E94AB0860E870E08FE0D7
:1015700093E00E947F1C88E291E09A838983AE0108
:101580004F5F5F4F60E070E0C7010E949417182F13
:1015900060E870E082E093E00E947F1C60E870E009
:1015A000812F0E94AB0860E870E08FEF92E00E940C
:1015B0007F1C60E870E08FEE92E00E947F1C81E06B
:1015C000D70157968C9321C085EE92E00E947F1C34
:1015D0000AC0F601918280820E949D1C04C00E9474
:1015E000A31C01C011ED812F0E94A91CD701ED9110
:1015F000FC910480F581E02DC7010995512E05C0AD
:1016000099ED592E02C084ED582E852DEB960FB61C
:10161000F894DEBF0FBECDBFDF91CF911F910F9128
:10162000FF90EF90DF90CF90BF90AF909F908F9002
:101630007F906F905F904F903F902F900895EF9222
:10164000FF920F931F93CF93DF937C018B01CCE02C
:10165000D0E0C7010C2E02C0959587950A94E2F759
:10166000982F9F7080E3890F8A3310F087E3890FEA
:10167000B8010E94721C2497CC3F8FEFD80749F71E
:10168000DF91CF911F910F91FF90EF900895AF924E
:10169000BF92CF92DF92EF92FF920F931F93CF935F
:1016A000DF93CDB7DEB762970FB6F894DEBF0FBEFB
:1016B000CDBFDC0157962C91222381F06C010E9452
:1016C000570DF6010389148925893689DC01CB0180
:1016D000801B910BA20BB30BB7FF02C0F12C05C10D
:1016E00061E870E086ED92E00E947F1C61E870E0A6
:1016F00080E090E00E941F0B61E870E083ED92E0D3
:101700000E947F1C61E870E080EA92E00E947F1CEA
:1017100061E870E0D6011A968C910E94AB0861E8EE
:1017200070E08DE992E00E947F1C61E870E086E63F
:1017300092E00E947F1C61E870E0F60183850E94C0
:10174000AB0861E870E083E692E00E947F1CD6015E
:101750001B968C911B9790E09A8B898BE12C8E01C4
:101760000F5F1F4F9E012F5E3F4F1A964C911A97A5
:1017700016966C91169714968D919C9115970E94D0
:101780000E16F82E882329F0F4E0FF1609F478C02D
:1017900006C029893A892330310508F055C061E82F
:1017A00070E081E592E00E947F1C61E870E08F2D7F
:1017B0000E94AB0861E870E08EE492E00E947F1C1A
:1017C000F1105EC089899A89892B09F459C060E8B3
:1017D00070E08DE292E00E947F1CA988BA880CE03C
:1017E00010E0C501002E02C0969587950A94E2F795
:1017F000982F9F7080E3890F8A3318F560E870E0B6
:101800000E94721C045011090C3F8FEF180749F712
:1018100060E870E08AE292E00E947F1C60E870E07D
:1018200083E192E00E947F1C60E870E080E090E03D
:101830000E941F0B60E870E080E192E00E947F1C34
:101840002EC087E3890FDACFD6011D968D919C912A
:101850001E97009721F1DC01ED91FC910190F08140
:10186000E02D8E010F5F1F4F40E0B601099517C0B4
:10187000232B31F060E870E08BE092E00E947F1C47
:101880000E94570DF601208DDC01CB01820F911DC6
:10189000A11DB11D838B948BA58BB68B26C0898926
:1018A0009A89892B69F38091000190910101803818
:1018B000910534F310E029893A89812F90E082174D
:1018C0009307B0F6E1E0F0E0EC0FFD1FE80FF91F21
:1018D00060E870E080810E94AB0860E870E08EE014
:1018E00092E00E947F1C1F5FE6CF8F2D62960FB69D
:1018F000F894DEBF0FBECDBFDF91CF911F910F9146
:10190000FF90EF90DF90CF90BF90AF9008958CE460
:1019100092E00E94D80E40E06CE472E082E392E034
:101920000E94A90740E06CE472E088E192E00E9426
:10193000A90740E06CE472E08EEF91E00E94A907F5
:1019400040E06CE472E084EE91E00E94A90782E539
:1019500091E09093D9018093D8019093CD01809329
:10196000CC019093C1018093C0019093B501809305
:10197000B4016CE472E083EA91E00E94C71A6CE45F
:1019800072E082E991E00C94C71AAF92BF92CF92B5
:10199000DF92EF92FF920F931F93CF93DF937C011F
:1019A000CB01D22EDB01ED91FC910084F185E02D7D
:1019B00009951F928F938BEE93E09F938F930E94D4
:1019C0001804E8015801AD0CB11C0F900F900F9056
:1019D0000F9085EEC82E83E0D82ECA15DB0561F086
:1019E00089911F928F93DF92CF920E9418040F90DB
:1019F0000F900F900F90F1CF82EE93E09F938F9313
:101A00000E9418040F900F90F8018281813049F4F0
:101A100088EC93E09F938F930E9418040F900F908F
:101A20000FC0D701129688E0F80101900D928A95B7
:101A3000E1F70E94570DD7011B967C936E931A977E
:101A4000DF91CF911F910F91FF90EF90DF90CF909A
:101A5000BF90AF90089580E090E008958FEF9FEFE2
:101A6000089581E090E008950895862F0E941F1D3B
:101A700081E090E00895FB0180810E941F1D81E0BC
:101A800090E00895ECECF2E01382128288EE93E08D
:101A9000A0E0B0E084839583A683B78388E591E0D6
:101AA000918380838FEF9FEF9587848708950C94AF
:101AB000BC0D8F929F92AF92BF92CF92DF92EF9226
:101AC000FF920E94B1324B015C0120E030E04AE716
:101AD00055E40E9468336B017C0120E030E040E86F
:101AE0005FE30E947D3287FD24C020E03FEF4FE797
:101AF00057E4C701B6010E9463331816ACF420E026
:101B000030E040E251E4C501B4010E9468330E9414
:101B1000823220E931E06115710581F0C901019738
:101B2000F1F761507109F7CFC701B6010E94823207
:101B300002C061E070E0CB010197F1F7FF90EF90F8
:101B4000DF90CF90BF90AF909F908F90089582E0EC
:101B500084BD93E095BD9AEF97BD80936E00089584
:101B60002FB7F89480911C0390911D03A0911E0340
:101B7000B0911F032FBF08952FB7F89460911C03F5
:101B800070911D0380911E0390911F032FBF089534
:101B90009C014FB7F89480911C0390911D03A09174
:101BA0001E03B0911F034FBF821B930B08957894BF
:101BB0001F920F920FB60F9211248F939F93AF93A2
:101BC000BF9380911C0390911D03A0911E03B091BF
:101BD0001F030196A11DB11D80931C0390931D034B
:101BE000A0931E03B0931F03BF91AF919F918F915C
:101BF0000F900FBE0F901F901895CF93DF93FC01AD
:101C0000862F8078A9F4283008F04DC0442321F0B5
:101C10009581973009F447C0EF01A1E0B0E09D85C0
:101C2000992341F011962596A031B105C1F73BC02B
:101C300080E039C061111CC085E08A9FE0018B9F64
:101C4000D00D1124CE0FDF1F442331F081E48887AB
:101C500085818F5F858302C081E0888725E02A9F88
:101C6000C0012B9F900D1124E80FF91F80851BC028
:101C70006770660F660F660F442341F060648581CC
:101C80008F5F85838770687F682B03C02770687BB0
:101C9000622B25E02A9FC0012B9F900D1124E80F95
:101CA000F91F6087862FDF91CF910895611102C0DF
:101CB00006960895FC0121E03585631739F02F5F02
:101CC00035962031C9F780E090E00895069635E01A
:101CD000239F800D911D11240895DF92EF92FF92B2
:101CE0000F931F93CF93DF93EC01E62EF12C85E049
:101CF000689FB0011124FE01E60FF71F8085182FA1
:101D0000177086FF17C001E085E0D82EFE01D09E37
:101D1000E00DF11D11248085869586958695877046
:101D20001817F9F00F5F003189F78D81811302C018
:101D300011501D8385E08E9DF0018F9DF00D1124C3
:101D4000EC0FFD1F108681E0818712862296D783D3
:101D5000C683DF91CF911F910F91FF90EF90DF909D
:101D60000895602FCE010E946D0ED0CFFC0161342A
:101D700099F49C01255B3F4F61E0AC014E5F5F4FE2
:101D8000158666871786548743873596E217F307CB
:101D9000B9F7FC011582089521E03585631729F014
:101DA0002F5F35962031C9F70895622F0C946D0E80
:101DB000FC018AE691E0918380831582108681E0A0
:101DC00081871286CF01029697838683128228E04C
:101DD00023832CE32483DF019F01255B3F4F41E0F8
:101DE0001D961C921D971E964C931E971F961C9233
:101DF0001F971C969C938E931B971596A217B3075B
:101E000079F7EA58FF4F108281E180932403089507
:101E1000809124030895CF93C42F0E94560E0097FB
:101E200089F0DC01ED91FC911197309759F01396F0
:101E30009C9180E0891731F020812C1731F0339686
:101E40008F5FF8CF80E090E001C0CF01CF9108957F
:101E50000F931F93CF93DF932115310571F0E901A3
:101E6000042F162F0E94560EFC01892B41F012837D
:101E7000D183C083038380E003C088ED01C086ED79
:101E8000DF91CF911F910F910895CF92DF92FF9232
:101E90000F931F93CF93DF93662381F1F62E8C016E
:101EA0006C0186E5C80ED11CC0E0D0E0D6018D9152
:101EB0009D916D010097F1F0DC01ED91FC910084A2
:101EC000F185E02D0995F81215C0AB96CC0FDD1FFA
:101ED000C00FD11F88819981DC01ED91FC910480B4
:101EE000F581E02DDF91CF911F910F91FF90DF9051
:101EF000CF9009942196C031D105C1F680E0DF91E1
:101F0000CF911F910F91FF90DF90CF9008952E9861
:101F10000895CF93C82F0E94870FCEBD0DB407FE42
:101F2000FDCF1EBC0DB407FEFDCF0E94E3078EB5AA
:101F3000CF910895CF93DF93C82FD62F0E94870F9C
:101F4000C260CEBD0DB407FEFDCFDEBD0DB407FEF1
:101F5000FDCFDF91CF910C94E3078F929F92AF92C8
:101F6000BF92CF92DF92EF92FF920F931F93CF9386
:101F7000DF93EC01D62EC42E59010E94560E7C012F
:101F8000009709F445C0FC0180819181892B09F4F7
:101F900041C04C2D6D2DCE010E940B0FF501918398
:101FA00080830097C9F1FC0182818695869590E037
:101FB0008031910514F08FE090E041E050E060E066
:101FC00070E04A015B0104C0880C991CAA1CBB1C70
:101FD0008A95D2F7D501C4010197F80191838083D6
:101FE0006D2D80EE0E949A0F88ED0E94890FF701F7
:101FF0009481992331F0CA58DF4F68816260682B61
:1020000002C0682F697F88ED0E949A0F80E005C0AA
:1020100086ED03C087ED01C08BEDDF91CF911F915D
:102020000F91FF90EF90DF90CF90BF90AF909F9077
:102030008F9008958F929F92AF92BF92CF92DF922E
:10204000EF92FF920F931F93CF93DF93862E942EE0
:1020500059010E94570D6B017C0128E8C20E23E153
:10206000D21EE11CF11C00E010E0D0E0C0E0982896
:102070000E94570DDC01CB018C199D09AE09BF09E7
:10208000B7FF2DC0692D80EF0E949A0F0E94570D57
:10209000DC01CB018C199D09AE09BF09B7FF09C04E
:1020A00088EC0E94890F87FFF1CF60E888EC0E94DE
:1020B0009A0F88EF0E94890FC82FCF70C43019F093
:1020C000CE3051F00CC00F5F1F4FA114B10481F24C
:1020D0000A151B0569F603C0DF5FD33049F68C2F64
:1020E000DF91CF911F910F91FF90EF90DF90CF90F4
:1020F000BF90AF909F908F9008959F92AF92BF92A4
:10210000CF92DF92EF92FF920F931F93CF93DF93C3
:102110007C01D42F122F902E00E06C01C60ED11C32
:10212000C60ED11C86E5C80ED11CA42EB12CABE284
:10213000AA0EB11CAA0CBB1CAE0CBF1CF601808100
:102140009181DC01ED91FC910280F381E02D292D3C
:10215000412F6D2F0995803EC9F4D1110BC061E06C
:1021600088EE0E949A0F66E670E080E090E00E94A0
:10217000590D14C0F50180819181DC01ED91FC9134
:102180000284F385E02D612F099508C08D3021F47C
:10219000033008F03FC014C081113FC0F6018081B8
:1021A0009181DC01ED91FC910190F081E02D292DD0
:1021B000412F6D2F0995C82F8D3051F4033050F405
:1021C00064E670E080E090E00E94590D0F5FB6CFAA
:1021D000882311F1D1110BC061E088EE0E949A0FA3
:1021E00066E670E080E090E00E94590D11C0ED2F8E
:1021F000F0E0BB96EE0FFF1FEE0DFF1D8081918179
:10220000DC01ED91FC910284F385E02D612F0995AD
:102210008C2F03C08DE001C080E0DF91CF911F9132
:102220000F91FF90EF90DF90CF90BF90AF909F9075
:1022300008950F931F93CF93DF93182F062FEA0172
:102240000E94870F12601EBDFE01802F882339F087
:102250000DB407FEFDCF91919EBD8150F7CFC00F09
:10226000D11D0DB407FEFDCF0E94E307CE01DF9123
:10227000CF911F910F9108952F923F924F925F92AD
:102280006F927F928F929F92AF92BF92CF92DF9286
:10229000EF92FF920F931F93CF93DF9300D000D064
:1022A0001F92CDB7DEB77B014A016901FB01F181C5
:1022B000F9838F2F8150803408F074C00E94570D2D
:1022C0002B013C0128E8420E23E1521E611C711CC7
:1022D000F701828180FD02C060E401C060E888EE01
:1022E0000E949A0F312C9981892F90E09A838983DB
:1022F000C114D10409F449C0E981FA81FD83EC835A
:10230000CE16DF0610F4DD82CC82FC81FB83A801AF
:102310006F2F80E10E9419116C8188E30E949A0F4F
:10232000F7016081606280EF0E949A0F88EC0E9442
:10233000890F87FFFBCF60E888EC0E949A0F88EF37
:102340000E94890F8F70382EA12CB12C212C3320A4
:1023500009F45AC00E94570DDC01CB01841995097C
:10236000A609B709B7FF50C01FC02EE0321609F406
:1023700046C084E0381209C0FFEFAF1ABF0A8114CB
:102380009104D9F0A814B904C1F488EF0E94890F10
:1023900085FB882780F9F701928180FB90F9928371
:1023A000832D39C08AED37C0F6E03F12DECF60E8FA
:1023B00070E085EF93E00E947F1C60E088E30E945C
:1023C0009A0FF801608180E10E949A0F6B8188E387
:1023D0000E949A0FF7016081606280EF0E949A0F5D
:1023E00088EC0E94890F87FFFBCF60E888EC0E9491
:1023F0009A0F88EF0E94890F8F70382EA8CF2394F0
:1024000023E02212DACFC1CFEC81FD81CE1ADF0AA0
:102410000E0F1F1F6DCF0F900F900F900F900F900A
:10242000DF91CF911F910F91FF90EF90DF90CF90B0
:10243000BF90AF909F908F907F906F905F904F90E4
:102440003F902F9008952F923F924F925F926F92FC
:102450007F928F929F92AF92BF92CF92DF92EF9234
:10246000FF920F931F93CF93DF93CDB7DEB72A97D9
:102470000FB6F894DEBF0FBECDBF9D838C836B017A
:102480005F834E835901EA82F90180809180FB01CC
:10249000F181FB83F90111821082FB01828181FDB0
:1024A00002C060E101C060E288EE0E949A0FFA81EA
:1024B0004F2E512C612C712C88862E813F81F60184
:1024C000408160E08C819D810E941A108983863052
:1024D00039F460E870E089EF93E00E947F1CEDCF53
:1024E000F981F11163C088EC0E94890F82FF5CC002
:1024F00080E30E94890F382E90E08816990608F430
:102500003884F501808191819401281B390B3A8729
:10251000298737FF02C01A861986E32CF12C89859A
:102520009A85E816F90614F4FA86E98629840E9449
:10253000870F98E09EBD0DB407FEFDCFF801222065
:1025400041F01EBC2A940DB407FEFDCF8EB58193D9
:10255000F6CFE985FA850E0F1F1F0E94E30764E09E
:1025600088EC0E949A0FF50180819181E80EF91E96
:10257000F182E082FB813F1618F0E814F90458F06C
:1025800088EF0E94890F82958170F601928180FB0D
:1025900091F992830BC0FA81FF2309F48ECFC30116
:1025A000B2010E94590D89CF20EF298389812A9693
:1025B0000FB6F894DEBF0FBECDBFDF91CF911F9154
:1025C0000F91FF90EF90DF90CF90BF90AF909F90D2
:1025D0008F907F906F905F904F903F902F900895D5
:1025E0002F923F924F925F926F927F928F929F9223
:1025F000AF92BF92CF92DF92EF92FF920F931F9311
:10260000CF93DF93CDB7DEB761970FB6F894DEBFF7
:102610000FBECDBF3C01F42E322E202EC98A4EA013
:102620005FA0C8A4D9A4188A1F861E861D868E01A5
:10263000035F1F4F9E01215F3F4F0E94AD0F81112D
:1026400096C039822A82EB8289898C83BE82AD82D0
:1026500098868F82AE014F5F5F4F68E080E20E94F4
:1026600019112D853E854F2D60E1C3010E941A107E
:10267000182F811178C0932D9078392EC114D10470
:1026800009F462C060E870E0992309F447C085E767
:1026900094E00E947F1CEF85F889828182608283AA
:1026A0005401A114B10409F454C05C864B864D85D5
:1026B0005E856F857889E12C86019E01255F3F4FFD
:1026C000C3010E942312182F863039F460E870E0AD
:1026D00081E794E00E947F1CE4CF811144C0AAA549
:1026E000BBA5109799F0ED91FC9111970190F081A5
:1026F000E02DC4018A199B099A8789876B857C859F
:102700009E01275F3F4FA601CD0109958B859C85D2
:10271000A81AB90A8415950520F616C08DE694E02E
:102720000E947F1C6F857889FB0182818160828392
:102730004D855E8586019201C3010E943C11811185
:1027400016C02D853E8511C02D853E85311005C0F2
:102750000CC0111108C02D853E8560EA4F2DC301C4
:102760000E941A1004C0812F02C060E8F7CF619662
:102770000FB6F894DEBF0FBECDBFDF91CF911F9192
:102780000F91FF90EF90DF90CF90BF90AF909F9010
:102790008F907F906F905F904F903F902F90089513
:1027A0008F929F92AF92BF92CF92EF920F931F930F
:1027B0001F921F921F930F933F932F934901A12CB8
:1027C000B12CCC24C394E12C06E020E80E94F01246
:1027D0000F900F900F900F900F900F901F910F91EF
:1027E000EF90CF90BF90AF909F908F9008958F9271
:1027F0009F92AF92BF92CF92EF92FF920F931F9250
:102800001F92FF92EF923F932F934901A12CB12C7D
:1028100022E0C22EE02E06E020E80E94F0120F9087
:102820000F900F900F900F900F900F91FF90EF90DF
:10283000CF90BF90AF909F908F9008954F925F92EE
:102840006F927F928F929F92AF92BF92CF92DF92C0
:10285000EF92FF920F931F93CF93DF93CDB7DEB725
:10286000C054D1090FB6F894DEBF0FBECDBF3C01F6
:10287000D62E542E422EC02ECE0101965C017C0134
:10288000022F29E030E0C3010E94F71381111BC021
:102890008B809C801F93CF92BF92AF921F9280E457
:1028A0008F93A12CB12C82E0C82EE42C06E020E806
:1028B000452D6D2DC3010E94F0120F900F900F90C7
:1028C0000F900F900F90C05CDF4F0FB6F894DEBFF3
:1028D0000FBECDBFDF91CF911F910F91FF90EF9071
:1028E000DF90CF90BF90AF909F908F907F906F9030
:1028F0005F904F9008958F929F92AF92BF92CF9228
:10290000EF920F93CF931F921F921F921F921F92CD
:102910001F92812C912CA12CB12CC12CE22E05E010
:1029200020E00E94F012C82F6CE271E080E090E09D
:102930000E94590D0F900F900F900F900F900F90D5
:102940008C2FCF910F91EF90CF90BF90AF909F9031
:102950008F9008950F931F93CF93DF938A3F3FEF9C
:10296000930711F486ED2DC0DC011696ED91FC91D4
:102970001797EF2B09F1122F242FEC011A8740E053
:102980000E94FD0D082F8823C9F0682FCE010E94F8
:10299000560E009739F3FC011483202F40E060E0CD
:1029A000CE010E947B14182F882351F0602FCE0196
:1029B0000E94B60E812F05C087ED03C084ED01C0D3
:1029C00080E0DF91CF911F910F9108952F923F9258
:1029D0004F925F926F927F928F929F92AF92BF922F
:1029E000CF92DF92EF92FF920F931F93CF93DF93DB
:1029F000CDB7DEB766970FB6F894DEBF0FBECDBF7A
:102A00001B8A38E03C8B3CE33D8B8A3F3FEF9307CA
:102A100009F464C0522E342E462E7C01DC01169639
:102A2000CD90DC901797CE01439617969C938E938A
:102A300016971A962C938E010F5F1F4F22E130E0FC
:102A400040E060E0C7010E94D013F701D782C68240
:102A50008111A6C089849A846B847C84FD81FE8B5D
:102A60002E80670136E5C30ED11C560110E0D5015A
:102A70008D919C910097F1F1DC01ED91FC91008426
:102A8000F185E02D0995811135C0F5018081918195
:102A9000DC01ED91FC910088F189E02D622D099512
:102AA000882341F1F50180819181DC01ED91FC9158
:102AB0000484F585E02DA301B4010995811110C0AE
:102AC000F50180819181DC01ED91FC910684F7850F
:102AD000E02D6E890995811103C00CC086ED60C0A0
:102AE000052D232D442D612FC7010E947D10813DAE
:102AF00009F056C01F5FB2E0AB0EB11C103109F0F7
:102B0000B6CF10E0F601808191810097E1F1DC0100
:102B1000ED91FC910084F185E02D0995811133C080
:102B2000F60180819181DC01ED91FC910088F189B1
:102B3000E02D622D09958823D9F0F60180819181DD
:102B4000DC01ED91FC910484F585E02DA301B40135
:102B50000995811118C0F60180819181DC01ED9108
:102B6000FC910684F785E02D6E89099581110BC0D3
:102B7000052D232D442D612FC7010E947D10982F14
:102B8000977F913D69F41F5FE2E0CE0ED11C1031BA
:102B900009F0B8CF252D432D642DC7010E94AA143A
:102BA00066960FB6F894DEBF0FBECDBFDF91CF9112
:102BB0001F910F91FF90EF90DF90CF90BF90AF905B
:102BC0009F908F907F906F905F904F903F902F904D
:102BD00008958F929F92AF92BF92CF92EF920F93F0
:102BE0001F921F921F921F921F921F92812C912C55
:102BF000A12CB12CC12CE22E09E020E00E94F012A1
:102C00000F900F900F900F900F900F900F91EF90EB
:102C1000CF90BF90AF909F908F9008957F928F92AA
:102C20009F92AF92BF92CF92DF92EF92FF920F935B
:102C30001F93CF93DF9300D000D0CDB7DEB76C01E8
:102C4000762EF42E590148011C821B821A821982A9
:102C50008E010F5F1F4F9E012D5F3F4F0E94AD0FF2
:102C6000182F8823A9F161E870E088E494E00E94BD
:102C70007F1C61E870E0812F0E94AB0861E870E082
:102C800085E494E00E947F1C61E870E083E294E0B8
:102C90000E947F1C61E870E0872D0E94AB0861E80C
:102CA00070E080E294E00E947F1C61E870E080E0C8
:102CB00094E00E947F1C61E870E08F2D0E94AB08B9
:102CC00061E870E08DEF93E00E947F1C812F09C0C6
:102CD00049815A816B817C8184019501C6010E94E2
:102CE00023120F900F900F900F90DF91CF911F91B3
:102CF0000F91FF90EF90DF90CF90BF90AF909F909B
:102D00008F907F900895AF92BF92CF92DF92EF9213
:102D1000FF920F931F93CF938C011D990EC088ECE7
:102D20000E94890F85FF05C0C8010E94FE0760E26E
:102D300001C060E088EC0E949A0F8091910181307F
:102D400039F040F0823079F0833079F5C1E00CC081
:102D500083E106C080912403807F803131F181E1DD
:102D60008093240322C0C0E080912403807F8031BF
:102D7000E9F40E94570DDC01CB0188539F4FAF4F00
:102D8000BF4F8093200390932103A0932203B0931D
:102D9000230380E28093240380ED0E94890F682F33
:102DA0006F7D80ED0E949A0F01C0C0E0780186E53A
:102DB000E80EF11C6801A6E7CA0ED11C5701F50107
:102DC000819191915F01009739F0DC01ED91FC91C7
:102DD0000680F781E02D0995AC14BD0481F7809140
:102DE0002403803409F447C050F4803221F1803349
:102DF000A1F1813109F08EC0F60110820AC081353F
:102E000009F464C0803809F476C0803509F082C0C6
:102E100045C0D7018D919D917D01009739F0DC016E
:102E2000ED91FC910480F581E02D0995EC14FD04F1
:102E300081F782E16DC00E94570D0091200310912F
:102E400021032091220330912303DC01CB01801B5D
:102E5000910BA20BB30BB7FD5DC080ED0E94890FF3
:102E6000682F606280ED0E949A0F61E088EE0E94F8
:102E70009A0F80E44DC088EE0E94890F80FD4AC001
:102E800060E488EC0E949A0F88ED0E94890F682FF9
:102E9000686088ED0E949A0F80E53AC088EC0E9435
:102EA000890F86FF37C081E5809324030E94570D68
:102EB000DC01CB014496A11DB11D809320039093AA
:102EC0002103A0932203B093230324C00E94570D33
:102ED000C0902003D0902103E0902203F0902303C0
:102EE000DC01CB018C199D09AE09BF09B7FD12C0E9
:102EF00080E8809324032C2F40E060E0C8010E940A
:102F0000E614882321F0823D29F080EA01C080E99F
:102F100080932403CF911F910F91FF90EF90DF904A
:102F2000CF90BF90AF9008958F929F92AF92BF9233
:102F3000CF92EF920F93CF93DF93CDB7DEB7C0540C
:102F4000D1090FB6F894DEBF0FBECDBF5F934F938C
:102F50009E012F5F3F4F3F932F931F9220E42F93AB
:102F600020E8822E912C5B0132E2C32EE12C06E098
:102F700021E840E0FC016681848195810E94F01285
:102F80000F900F900F900F900F900F90C05CDF4F3D
:102F90000FB6F894DEBF0FBECDBFDF91CF910F917A
:102FA000EF90CF90BF90AF909F908F9008958F92A9
:102FB0009F92AF92BF92CF92DF92EF92FF920F93C8
:102FC000A42EB12C1F921F92DF92CF92FF92EF920C
:102FD0004701C22EE02E09E021E2462FFC01668166
:102FE000848195810E94F0120F900F900F900F90A6
:102FF0000F900F900F91FF90EF90DF90CF90BF90C8
:10300000AF909F908F9008958F929F92AF92BF92B2
:10301000CF92EF920F93A62EB12C1F921F921F9268
:103020001F921F921F92812C912CC22EE42E0AE037
:1030300021E240E0FC016681848195810E94F012CA
:103040000F900F900F900F900F900F900F91EF90A7
:10305000CF90BF90AF909F908F9008958F929F9246
:10306000AF92BF92CF92EF920F93A62EB12C1F92E8
:103070001F921F921F921F921F92812C912CC12C84
:10308000E42E0BE021E240E0FC0166818481958121
:103090000E94F0120F900F900F900F900F900F90D2
:1030A0000F91EF90CF90BF90AF909F908F90089529
:1030B000FC018285089581E0693009F080E008957F
:1030C000CF93DF93EC018A819B81DC01ED91FC9130
:1030D0000480F581E02D6A8509958A85813439F46B
:1030E000EA81FB81EA58FF4F80818B7F80831A86BB
:1030F0001B861C861D861E861F86188A80E0DF912F
:10310000CF9108958F929F92AF92BF92CF92EF92FC
:103110000F93A42EB12CB22A1F921F921F921F92BE
:103120001F921F92812C912CC12CE62E01E023E2EC
:1031300040E0FC016285828193810E94F0120F9031
:103140000F900F900F900F900F900F91EF90CF90E6
:10315000BF90AF909F908F9008958F929F92AF9263
:10316000BF92CF92EF920F93A62EB12C1F921F9277
:103170003F932F935F934F934A01C12CE12C00E0C2
:1031800023EA40E0FC016285828193810E94F01273
:103190000F900F900F900F900F900F900F91EF9056
:1031A000CF90BF90AF909F908F9008958F929F92F5
:1031B000AF92BF92CF92EF920F93A42EB12CB22A6E
:1031C0001F921F921F921F921F921F92812C912C6F
:1031D000C12CE62E03E023E240E0FC0162858281FF
:1031E00093810E94F0120F900F900F900F900F900C
:1031F0000F900F91EF90CF90BF90AF909F908F90D6
:1032000008952F923F924F925F926F927F928F928A
:103210009F92AF92BF92CF92DF92EF92FF920F9365
:103220001F93CF93DF93CDB7DEB7E9970FB6F8942E
:10323000DEBF0FBECDBFDC011A96DC90D11017C1E6
:10324000122FC42E69AF3C01FC01A280B380D501CE
:10325000ED91FC910190F081E02D60E0C5010995B0
:103260007C01009709F406C1FC01808091808114E3
:10327000910409F402C11301F4E02F0E311CDC01AA
:1032800011963C922E9214961C93FE0131962F01BA
:103290008F0128E030E040E060E0D30112968D918C
:1032A0009C9113970E94D013F70114828111EEC0F4
:1032B0008D81893009F0E4C01981D501ED91FC912F
:1032C0000280F381E02D2C2D41E069ADC501099507
:1032D000F3018287882309F4D6C098859583282F27
:1032E00040E060E0828193810E947B14C82E882395
:1032F00091F0D7018D929C92D501ED91FC910480C3
:10330000F581E02DD3011A966C91C5010995F30161
:103310001286DC2CBFC0212F113208F020E2D70129
:103320008D929C9221110CC0910142E0F3016285C3
:10333000828193810E94280FF82E811190C011C0C4
:1033400030E0820140E0D3011A966C911A971296F0
:103350008D919C9113970E94D013F82E81117FC0FC
:10336000E3CF1F921F925F924F921F9288E08F933C
:1033700058E0852E912CA12CB12C69E2C62EE12CAF
:1033800006E020EA40E0F3016285828193810E9499
:10339000F012F82E0F900F900F900F900F900F904B
:1033A00081115DC08B81D3011B968C931B97720199
:1033B00000E028E030E040E01A966C911A971296EF
:1033C0008D919C9113970E94F713F82E811147C09D
:1033D0002B813C81720140E0F301628582819381FF
:1033E0000E94F713F82E81113AC0298130E0CE01F6
:1033F00081967C0140E0D3011A966C911A9712963F
:103400008D919C9113970E94F713F82E811127C07C
:103410002E8140E0F3016285828193810E94E9154B
:10342000F82E81111CC011E0D3011B968C918117DD
:1034300040F020E0412F68E0C3010E94D6181F5FD2
:10344000F3CFD3011296ED91FC911397EA58FF4FF9
:1034500080818460808381E050968C931BC060E8FB
:1034600070E089E794E00E947F1CDF2C13C049EDD7
:10347000D42E10C036EDD32E0DC027EDD22E0AC0AB
:1034800091EDD92E07C084EDD82E04C0F7019182AA
:103490008082D82E8D2DE9960FB6F894DEBF0FBE30
:1034A000CDBFDF91CF911F910F91FF90EF90DF90F3
:1034B000CF90BF90AF909F908F907F906F905F90D4
:1034C0004F903F902F900895CF92DF92FF920F93ED
:1034D0001F93CF93DF9300D000D0CDB7DEB78C0120
:1034E000F62E19821A821B821C8220E0462F61E18F
:1034F0000E94821820E04F2D60E1C8010E948218CE
:1035000020E04F2D64E0C8010E94D61883E0C82E49
:10351000D12C9E012F5F3F4F44E050E06F2DC8013A
:103520000E94AD188823F1F020E04F2D64E1C8011E
:103530000E94821820E04F2D60E1C8010E9482188D
:1035400064E170E080E090E00E94590D0F900F90D0
:103550000F900F90DF91CF911F910F91FF90DF900F
:10356000CF90089589819A81AB81BC819D7F833002
:103570009140A041B105C1F264E670E080E090E0C6
:103580000E94590D81E0C81AD10819F6CDCFFC016F
:1035900084E791E09183808373836283128613862C
:1035A0001486158616861786108A148288E085830D
:1035B0009CE3968391E09783808784E081876115FF
:1035C0007105B1F0DB01AA5ABF4F80E090E02D9168
:1035D0003D91232B49F48B96880F991FDB01A80F8F
:1035E000B91FED93FC93089501968031910579F709
:1035F0000895EF92FF920F931F93CF938C01C62FE4
:103600007A01FA0180819181A281B3818130F3E056
:103610009F07F1E0AF07B105D1F060F48115E1E05B
:103620009E07AE07B10571F181309140A140B1050F
:1036300071F064C0833021E0920720E1A207B10558
:10364000E1F183309340A041B105B9F157C08091B9
:103650002503811153C020E04C2F61E1C8010E9475
:10366000821820E04C2F60E1C8010E94821820E0FF
:103670004C2F64E0C8010E94D61881E08093250396
:1036800081EB3DC020E0462F61E1C8010E94821815
:1036900020E04C2F60E1C8010E948218109225039F
:1036A000F80162856770C770660F660F660F6C2B36
:1036B000828193810E94450F21C020E04C2F64E15C
:1036C000C8010E94821820E04C2F60E1C8010E94CE
:1036D000821864E170E080E090E00E94590DF801EA
:1036E0006285F70121812695217067704C2FF801C2
:1036F000828193810E94E6141092250380E0CF918D
:103700001F910F91FF90EF900895CF92DF92EF926B
:103710000F931F93CF93DF93CDB7DEB72E970FB6DE
:10372000F894DEBF0FBECDBF6C0181E090E09E87B4
:103730008D87E12C8E010F5F1F4F9E01235F3F4F4E
:1037400041E0F6016285828193810E940E1681110B
:1037500051C002E011E089818023D1F019861A86D8
:103760001B861C869E01275F3F4F44E050E0612F7F
:10377000C6010E94AD1881110BC0AE01475F5F4FBB
:10378000612FC6010E94F91A813B99F1811132C063
:10379000000F1F5F1830F9F611E0F60183858117DD
:1037A00040F119861A861B861C869E01275F3F4FB3
:1037B00044E050E0612FC6010E94AD18811117C08E
:1037C00089859A85877091708130914081F48B85CD
:1037D0009C8581609C878B87AE01475F5F4F612F1F
:1037E000C6010E94F91A813B21F0811103C01F5FBD
:1037F000D4CF80E02E960FB6F894DEBF0FBECDBFBB
:10380000DF91CF911F910F91EF90DF90CF900895AE
:103810000F931F93CF93DF93FC012089211102C0E6
:1038200080E020C0EC010E94570D0C851D852E857F
:103830003F85DC01CB01801B910BA20BB30BB7FDC5
:10384000EFCFCE010E94851B182F0E94570DDC017F
:10385000CB018C599F4FAF4FBF4F8C879D87AE8751
:10386000BF87812FDF91CF911F910F910895CF9343
:10387000DF93FC01EB0180819181892B39F560E8B0
:1038800070E083E894E00E947F1C24C0DA012D914F
:103890003C91232BF9F0A881B9819C91A381B0E0E0
:1038A000A81BB10920813181A20FB31F9C93828193
:1038B00081508283DA018D919C91119701978D93AC
:1038C0009C93888199810196998388838281811153
:1038D000DDCF02C080E003C08381828381E0DF917D
:1038E000CF910895209100013091010126173707EB
:1038F0002CF0682F8CEC92E00C94CE1C08950F9362
:103900001F93CF93DF93209100013091010126177F
:10391000370774F0009761F08B01FC018491EF018F
:103920002196882329F0B8010E94721CFE01F6CF6F
:10393000DF91CF911F910F91089560E870E08BEABD
:1039400094E00C947F1C60E870E080EA94E00C94B2
:103950007F1CCF93C82F282F30E084E03595279522
:103960008A95E1F780E3820F8A3310F087E3820FB4
:1039700060E870E00E94721CCF7080E38C0F8A3385
:1039800010F087E38C0F60E870E00E94721C60E822
:1039900070E08DE994E0CF910C947F1CDC01ED91F7
:1039A000FC910190F081E02D0994809132040895FA
:1039B00008950895CF93DF932091AC05243049F505
:1039C00021E02093E90021E8215059F03091E800EE
:1039D00035FD07C0EFE3F1E03197F1F700C00000DB
:1039E000F3CF2091E80025FF14C0EC0140E050E047
:1039F00068E070E00E94AE208091E8008E778093AE
:103A0000E80088E0FE01AAE2B4E001900D928A95F8
:103A1000E1F7DF91CF910895CF93C0912803C111B1
:103A20000BC00E94BC0D643C79408105910520F0DB
:103A300081E080932803C1E08C2FCF910895FF92FD
:103A40000F931F93CF93DF93D82F0FB607FE83C03A
:103A50008091AC05843081F08091050190E0019661
:103A60002091070130E0822393232091060130E06A
:103A70008217930709F0CDC00E940C1D811110C060
:103A80008091050190E001962091070130E08223AA
:103A900093232091060130E08217930709F0B9C003
:103AA0000E94B00D8C01C091E900CF709091EC00A4
:103AB000892F817090FD80E8C82B82E08093E90017
:103AC00085E0F82E8091EB0085FD42C08091EB00EF
:103AD00080FF3EC08091EE0087FF3AC080910601D2
:103AE00090910501981709F457C09091E80095FF4F
:103AF0008EC0E0910301F0910401E80FF11D2081D7
:103B00008F5F909107018923809306012093F10034
:103B10008091E80085FDE2CF8091E80080FFDECF54
:103B20008091E8008E778093E800F0920201D6CF72
:103B30008091050190E001962091070130E08223F9
:103B400093232091060130E08217930709F44CC0BB
:103B5000CF70C093E90040910501842F90E0019659
:103B60002091070130E0822393232091060130E069
:103B70008217930709F450C0E0910301F09104010A
:103B8000E40FF11DD083809105018F5F90910701B3
:103B900089238093050140C08091E80085FF37C0EC
:103BA000D093F10021E03091F3008091F20090E099
:103BB000932B892B91F08091E80080FF0EC08091BB
:103BC000E80085FF03C01092F100F9CF8091E80072
:103BD0008E778093E800F0920201222309F4A8CFA7
:103BE000CF70C093E90018C080910201882309F4C6
:103BF000AFCF0E94B00D9C018017910711F489018D
:103C000061CF90910201915090930201F8CF20E092
:103C1000CACF40910501B0CF80E0DF91CF911F91D5
:103C20000F91FF90089508958091AB05811104C014
:103C30000E941A230C94772308951092AB050895DF
:103C4000089542E061EC81E00E94272042E261ECAD
:103C500082E00C9427208091AE05833009F453C094
:103C600030F4813071F0823009F48CC008958A30CC
:103C700009F478C08B3009F45EC0893009F09AC02D
:103C800020C08091AD05813A09F094C08091E80090
:103C9000877F8093E8008091B1059091B205892BD0
:103CA00021F468E08AE294E003C060E080E090E004
:103CB00070E00E94FB208091E8008B778093E80001
:103CC00008958091AD05813209F074C08091B105ED
:103CD0009091B205892B09F06DC08091E800877F33
:103CE0008093E8008091E80082FD05C08091AC05DA
:103CF0008111F8CF5FC08091F100809332048091F0
:103D0000E8008B7753C08091AD05813A09F052C02D
:103D10008091B1059091B205892B09F04BC080913B
:103D2000E800877F8093E8008091E80080FFFCCF67
:103D30008091120136C08091AD058132D9F5809114
:103D4000B1059091B205892BA9F58091E800877F94
:103D50008093E8000E945C208091AF05809312015F
:103D60000C9496278091AD05813221F58091E80071
:103D7000877F8093E8000E945C208091B00580934B
:103D8000330408958091AD05813AA1F48091E80053
:103D9000877F8093E8008091E80080FFFCCF8091CE
:103DA00033048093F1008091E8008E778093E800DF
:103DB0000C945C2008958091320480932903109222
:103DC00032040E94F1250C9496270C94DB1E0E946D
:103DD0004831809129038093320408950C94E71EA2
:103DE00008950C94F01E0C94F01ECF9384B7877F37
:103DF00084BF0FB6F894A895809160008861809385
:103E00006000109260000FBE90E080E80FB6F8945A
:103E100080936100909361000FBE8FE19DE10E944D
:103E2000EF3088E091E00E947E248EED94E00E94C5
:103E30007F030E94F31E0E9432250E941A230E94D3
:103E4000772378940E9434258091AC05843029F042
:103E50000E9463240E94F01EF7CF8CEC94E00E9435
:103E60007F030E94F11E8AEB94E00E947F03C2E070
:103E70008091AC05853019F40E949A07F9CF0E9411
:103E800038252091E4003091E5008091260390913F
:103E900027032817390709F468C08091E40090913E
:103EA000E50090932703809326030E940C1D88232E
:103EB00009F45BC08091AC05843009F056C0809154
:103EC000E9008F702091EC00922F917020FD90E816
:103ED000892BC093E9009091EB0090FF43C0909133
:103EE000EE0097FF3FC09091060120910501291730
:103EF00009F12091E80025FF1DC0E0910301F09138
:103F00000401E90FF11D30819F5F20910701922389
:103F1000909306013093F1009091E80095FDE3CF76
:103F20009091E80090FFDFCF9091E8009E7790930A
:103F3000E800D9CF9091F3002091F20030E0392BC6
:103F4000232B81F09091E80090FF0CC09091E80045
:103F500095FF03C01092F100F9CF9091E8009E7791
:103F60009093E8008F708093E9000E94632480CFD3
:103F7000292F332723303105C9F060F42130310572
:103F800081F02230310509F044C082E490E026E45B
:103F900035E043C021323105E1F02232310549F1EB
:103FA00038C082E190E028E835E037C099278130B9
:103FB000910549F028F0029761F5E4EFF4E005C0BF
:103FC000E2E4F5E002C0E2E3F5E0849190E09F01D5
:103FD00024C06115710541F061307105D1F489E0AB
:103FE00090E021E735E019C089E090E028E535E070
:103FF00014C06115710541F06130710551F482E220
:1040000090E02AE935E009C080E490E02CEB35E04F
:1040100004C080E090E020E030E0FA0131832083AA
:10402000089580E189BD82E189BD09B400FEFDCF1C
:104030008091D8008F7D8093D8008091E0008260CD
:104040008093E0008091E00081FDFCCF0895982FDF
:10405000973068F59093E900981739F07091EC006B
:104060002091ED005091F00003C0242F762F50E0F6
:1040700021FD02C09F5FECCF3091EB003E7F30937B
:10408000EB003091ED003D7F3093ED003091EB007F
:1040900031603093EB007093EC002093ED0050936F
:1040A000F0002091EE0027FDE5CF80E008958F70AD
:1040B0008093E90081E008958091AD0587FF11C0EC
:1040C0008091E80082FD05C08091AC058111F8CF98
:1040D00011C08091E8008B770BC08091AC058823DC
:1040E00049F08091E80080FFF8CF8091E8008E775A
:1040F0008093E80008952091E4003091E50095E672
:104100004091EC00842F817040FF23C08091E80033
:1041100080FD1DC08091AC05882399F0853099F011
:104120008091EB0085FD11C04091E4005091E500C5
:104130002417350729F3915011F09A01E1CF84E05B
:10414000089582E0089583E0089581E0089580E075
:1041500008954091E80042FFDDCF0895CF92DF92AD
:10416000EF92FF920F931F93CF93DF93EC018B019C
:104170007A010E947B20811135C0E114F10439F0ED
:10418000F70180819181081B190BC80FD91FC12C21
:10419000D12C0115110529F18091E80085FD18C089
:1041A0008091E8008E778093E8000E946324E114F8
:1041B000F10449F0F70180819181C80ED91ED182A6
:1041C000C08285E00FC00E947B20882311F30AC0C3
:1041D00089918093F10001501109FFEFCF1ADF0A96
:1041E000D8CF80E0DF91CF911F910F91FF90EF909A
:1041F000DF90CF9008952091B3053091B405261734
:10420000370748F06115710539F42091E8002E77E1
:104210002093E80001C0B901FC0120E0611571059F
:1042200079F18091AC058823F1F18530F1F180912D
:10423000E80083FD3CC08091E80082FD2EC08091A3
:10424000E80080FFEBCF2091F3008091F20090E036
:10425000922B6115710551F08830910538F4219148
:104260002093F100615071090196F3CF21E0089786
:1042700009F020E08091E8008E778093E800CECFAF
:104280002111CFCF0AC08091AC05882361F0853021
:1042900061F08091E80083FD0AC08091E80082FF10
:1042A000F2CF80E0089582E0089583E0089581E0F0
:1042B00008952091B3053091B4052617370748F0CB
:1042C0006115710539F42091E8002E772093E800FC
:1042D00001C0B901FC0120E06115710591F18091E7
:1042E000AC05882309F440C0853009F43FC08091B3
:1042F000E80083FD3DC08091E80082FD2FC08091E1
:10430000E80080FFE9CF2091F3008091F20090E077
:10431000922B6115710559F08830910540F4249174
:104320002093F1003196615071090196F2CF21E09E
:10433000089709F020E08091E8008E778093E800EC
:10434000CBCF2111CCCF0AC08091AC05882361F07E
:10435000853061F08091E80083FD0AC08091E8001B
:1043600082FFF2CF80E0089582E0089583E008950F
:1043700081E008951F93CF93DF93CDB7DEB7AA975F
:104380000FB6F894DEBF0FBECDBFEDEAF5E0809129
:10439000F100819325E0E53BF207C9F70E942B1E4F
:1043A0008091E80083FF2EC18091AD059091AE050C
:1043B000492F50E04A30510508F024C1FA01EA5A69
:1043C000FF4F0C94D533803821F0823809F01AC1A0
:1043D00008C08091A9059091AA05992389F082606F
:1043E0000FC08091B1058F70873008F00BC18093AA
:1043F000E9008091EB0085FB882780F91092E900A5
:104400009091E800977F9093E8008093F1001092DC
:10441000F100D1C0282F2D7F09F0F4C0882319F0B6
:10442000823061F0EFC08091AF05813009F0EAC0C1
:10443000933009F080E08093AA052EC08091AF05EB
:1044400081112AC08091B1058F702FEF280F26307F
:1044500008F0D8C08093E9002091EB0020FF1CC039
:10446000933021F48091EB00806214C09091EB00B6
:1044700090619093EB0021E030E0A90102C0440F6D
:10448000551F8A95E2F74093EA001092EA00809166
:10449000EB0088608093EB001092E9008091E800C7
:1044A000877F8093E8000E945C20ACC08111AAC085
:1044B0001091AF051F778091E3008078812B809366
:1044C000E3008091E800877F8093E8000E945C20F1
:1044D0008091E80080FFFCCF8091E30080688093AA
:1044E000E300111102C082E001C083E08093AC05BB
:1044F00089C08058823008F085C08091AF059091C6
:10450000B0058C3D53E0950779F583E08A838AE214
:1045100089834FB7F894DE01139620E03EE051E224
:10452000E32FF0E050935700E49120FF03C0E295A1
:10453000EF703F5FEF708E2F90E0EA3010F0C7967B
:1045400001C0C0968D939D932F5F243149F74FBFD3
:104550008091E800877F8093E8006AE270E0CE01F6
:1045600001960E94FB2016C06091B1057091B205C2
:10457000AE014F5F5F4F0E94B81FBC01892B09F449
:1045800041C09091E800977F9093E80089819A81DB
:104590000E9459218091E8008B778093E80032C017
:1045A000803881F58091E800877F8093E8008091D2
:1045B000A8058093F1008091E8008E7772CF811179
:1045C00021C08091AF059091B00599270297D4F44E
:1045D0008091E800877F8093E8008091AF05809309
:1045E000A8050E945C208091A805811106C08091D9
:1045F000E30087FD02C081E001C084E08093AC0548
:104600000E94211E8091E80083FF0AC08091E8008B
:10461000877F8093E8008091EB0080628093EB00BD
:10462000AA960FB6F894DEBF0FBECDBFDF91CF9133
:104630001F9108950E9488230E949023E0EEF0E0ED
:10464000808181608083E8EDF0E080818F778083D6
:1046500019BCA7EDB0E08C918E7F8C9380818F7E0A
:1046600080831092AB0508950F931F93CF93DF9330
:104670000E9488230E949023C8EDD0E088818F7724
:10468000888388818068888388818F7D888319BC2E
:104690001092AC051092A8051092AA051092A905D7
:1046A00000EE10E0F80180818B7F8083888181603B
:1046B000888342E060E080E00E942720E1EEF0E0A5
:1046C00080818E7F8083E2EEF0E080818160808354
:1046D000808188608083F80180818E7F80838881DB
:1046E00080618883DF91CF911F910F910895E8ED4C
:1046F000F0E080818F7E8083E7EDF0E08081816053
:10470000808384E082BF81E08093AB050C943423E6
:10471000E8EDF0E080818E7F80831092E2000895C2
:104720001092DA001092E10008951F920F920FB6D6
:104730000F9211242F933F934F935F936F937F9327
:104740008F939F93AF93BF93EF93FF938091E1007B
:1047500082FF0BC08091E20082FF07C08091E100E0
:104760008B7F8093E1000E9462248091DA0080FFB9
:104770001FC08091D80080FF1BC08091DA008E7F1F
:104780008093DA008091D90080FF0DC080E189BD5F
:1047900082E189BD09B400FEFDCF81E08093AC05C4
:1047A0000E94141E05C019BC1092AC050E941D1E6B
:1047B0008091E10080FF19C08091E20080FF15C068
:1047C0008091E2008E7F8093E2008091E200806120
:1047D0008093E2008091D80080628093D80019BC59
:1047E00085E08093AC050E94E51E8091E10084FF86
:1047F00030C08091E20084FF2CC080E189BD82E15D
:1048000089BD09B400FEFDCF8091D8008F7D8093D3
:10481000D8008091E1008F7E8093E1008091E200DA
:104820008F7E8093E2008091E20081608093E200BD
:104830008091A805882311F084E007C08091E300EF
:1048400087FD02C081E001C083E08093AC050E9437
:10485000EE1E8091E10083FF24C08091E20083FF7F
:1048600020C08091E100877F8093E10082E0809307
:10487000AC051092A8058091E1008E7F8093E10045
:104880008091E2008E7F8093E2008091E20080615F
:104890008093E20042E060E080E00E9427200E94D6
:1048A000201EFF91EF91BF91AF919F918F917F91CA
:1048B0006F915F914F913F912F910F900FBE0F908D
:1048C0001F9018950895CF938091AC058823A1F08F
:1048D000C091E900CF709091EC00892F817090FD1C
:1048E00080E8C82B1092E9008091E80083FD0E94C7
:1048F000BA21CF70C093E900CF9108959093390405
:10490000809338040895E0913804F0913904309789
:1049100021F00190F081E02D099480E00895EF925C
:10492000FF920F931F93CF93DF93E0913804F091A0
:1049300039043097B1F18C010280F381E02D0995A3
:104940008091A60582FF2DC080FF04C082E296E020
:104950000E947F03E80118E08CE1E82E86E0F82E43
:104960008091A60580FF0BC088811F928F93FF92D4
:10497000EF920E9418040F900F900F900F9011501B
:1049800021961111EDCF8091A60580FF0AC08AE122
:1049900096E0DF91CF911F910F91FF90EF900C94D3
:1049A0007F03DF91CF911F910F91FF90EF900895BA
:1049B000CF93DF93209136043091370428173907BD
:1049C00009F19093370480933604E0913804F09114
:1049D00039043097B9F0EC010680F781E02D099594
:1049E0008091A60582FF0EC080FF0CC0DF93CF939D
:1049F0008CE096E09F938F930E9418040F900F9085
:104A00000F900F90DF91CF910895CF93DF93209176
:104A10003404309135042817390709F1909335048F
:104A200080933404E0913804F09139043097B9F060
:104A3000EC010084F185E02D09958091A60582FFA7
:104A40000EC080FF0CC0DF93CF938CEF95E09F9357
:104A50008F930E9418040F900F900F900F90DF918A
:104A6000CF9108950C94F2250E94A70D0C9489080B
:104A70008F929F92AF92BF92CF92DF92EF92FF926E
:104A80000F931F93CF93DF9300D000D01F92CDB729
:104A9000DEB70E9428060BE314E0F12C8F2D0E9454
:104AA00010074C01F801A080B180A826B926A114F6
:104AB000B10439F4F3940E5F1F4FF0E1FF12EECF13
:104AC00039C08091A60581FD0E943D07E12CCC24D0
:104AD000C394D12CC5018C219D21892B21F1E98220
:104AE000FA8221E0C4018C219D21892B09F420E068
:104AF0002B830E94B00D8160782F9D838C83498128
:104B00005A816B818D810E94F52549815A816B8183
:104B10007C818D810E94F530F801808191818C2506
:104B20009D2591838083E394CC0CDD1CF0E1EF1292
:104B3000D1CFC0CF8FEF89838A831B820E94B00DB3
:104B40008160782F9D838C8349815A816B818D810F
:104B50000E94F5250E94F4300E94832490913A042B
:104B6000891759F10E94832480933A049091A605F5
:104B700092FF0EC090FF0CC01F928F938DE296E0C3
:104B80009F938F930E9418040F900F900F900F9097
:104B900080913A040F900F900F900F900F90DF913B
:104BA000CF911F910F91FF90EF90DF90CF90BF902A
:104BB000AF909F908F900C9406310F900F900F90B4
:104BC0000F900F90DF91CF911F910F91FF90EF9079
:104BD000DF90CF90BF90AF909F908F9008950C94EE
:104BE0003E070895089508950895CF93DF93CDB7B4
:104BF000DEB72B970FB6F894DEBF0FBECDBF942F54
:104C00004F83252F588769877A878B874A855B85ED
:104C1000452B31F02F3F31F481E09F3F19F403C061
:104C200081E001C080E080FD07C04F815885698523
:104C30007A858B850E94F530DE01119686E0FD01B4
:104C400011928A95E9F785E0FE01379601900D9261
:104C50008A95E1F749815A816B817C818D819E81A2
:104C60000E94732D2B960FB6F894DEBF0FBECDBFFA
:104C7000DF91CF910895CF93DF93882309F4E8C0A3
:104C80009EE7980F933018F5823829F0833831F079
:104C9000C4E0D7E405C0C2E0D9E302C0C1E0D3E577
:104CA0000E9483248C2309F0D3C08D2F0E945130A1
:104CB0000E94C9302FEF81EE94E021508040904057
:104CC000E1F700C000008D2F0E946E3006C09CEFFF
:104CD000980F913A30F40E945130DF91CF910C94AB
:104CE000C93090E2980F983050F4877091E001C07D
:104CF000990F8A95EAF7892F0E948F30EECF9BE5B6
:104D0000980F933080F4853A29F0863A31F083E8A1
:104D100090E005C081E890E002C082E890E0DF9179
:104D2000CF910C94D82498E5980F973108F090C053
:104D3000883A09F445C0893A09F445C08A3A09F429
:104D400045C08B3A09F445C08C3A09F445C08D3A08
:104D500009F445C08E3A09F445C08F3A09F445C0BC
:104D6000813B09F445C0803B09F445C0823B09F40E
:104D700045C0833B09F445C0843B09F445C0853BED
:104D800009F445C0863B09F445C0873B09F445C09A
:104D9000883B09F445C0893B09F445C08A3B09F4C6
:104DA00045C08B3B09F445C08C3B09F445C08D3BA5
:104DB00009F445C08E3B09F445C080E090E044C052
:104DC00082EE90E041C089EE90E03EC08AEE90E035
:104DD0003BC085EB90E038C086EB90E035C083EBBC
:104DE00090E032C084EB90E02FC087EB90E02CC0C5
:104DF0008CEC90E029C08DEC90E026C083E891E037
:104E000023C08AE891E020C082E991E01DC084E9D6
:104E100091E01AC081E292E017C083E292E014C0F0
:104E200084E292E011C085E292E00EC086E292E058
:104E30000BC087E292E008C08AE292E005C08FE6EC
:104E400090E002C080E790E0DF91CF910C940525BF
:104E5000DF91CF910895CF93DF93882309F44FC05A
:104E60009EE7980F933000F5823829F0833831F0AF
:104E7000C4E0D7E405C0C2E0D9E302C0C1E0D3E595
:104E80000E9483248C23D9F18D2F0E9451300E94DF
:104E9000C9302FEF81EE94E0215080409040E1F73F
:104EA00000C000008D2F04C09CEF980F913A18F4B9
:104EB0000E946E300DC090E2980F983068F48770B1
:104EC00091E001C0990F8A95EAF7892F0E949530E9
:104ED000DF91CF910C94C9309BE5980F933030F45B
:104EE00080E090E0DF91CF910C94D824885A8731EC
:104EF00030F480E090E0DF91CF910C940525DF91B4
:104F0000CF910895882321F00E948F300C94C930EE
:104F10000895882321F00E9495300C94C93008959B
:104F20000E94AF300E947E300C94C9300E949F30A6
:104F30000C949027CF92DF92EF92FF920F931F93E2
:104F4000CF93DF9300D000D01F92CDB7DEB76C01B6
:104F50000E9408318111CDC285E0F601DE01119673
:104F600001900D928A95E1F7F601408151812381EC
:104F700034812115310531F05F3F31F481E04F3F3D
:104F800019F403C081E001C080E080FDB2C2F601E7
:104F9000F280E580E2948FE0E82249835A83FB8225
:104FA000722F3D832C836F2D8D810E94CD2F8C011C
:104FB0000E94CC2F0E94C62EE12FE295EF708E2F1B
:104FC00090E0FC01E05AFF4F0C94D533812F807F95
:104FD0001F70882311F01295107FFF20B9F0112364
:104FE00029F0812F0E94A2300E94C930802F0F909B
:104FF0000F900F900F900F90DF91CF911F910F9115
:10500000FF90EF90DF90CF900C943B26802F0E9472
:105010002B27112309F46DC2812F0E94A8300F9015
:105020000F900F900F900F90DF91CF911F910F91E4
:10503000FF90EF90DF90CF900C94C930812F807F4C
:105040001F70803211F01295107F002319F001308B
:1050500009F12BC0FF20A9F0EE2059F1F1E0812FDA
:10506000EF1228C00F900F900F900F900F90DF91CC
:10507000CF911F910F91FF90EF90DF90CF900C9404
:10508000B230EE2021F021E0E21609F432C20E9493
:10509000B5304DC0FF20E9F085E08E1508F429C237
:1050A0000E948C30812329F042C0FF20F1F1E110F1
:1050B00015C0812F0F900F900F900F900F90DF91E0
:1050C000CF911F910F91FF90EF90DF90CF900C94B4
:1050D000822794E09E1508F40CC229C0F601858150
:1050E00080FF13C08F708583E4CF003F09F43EC179
:1050F00008F00AC180E4800F803208F40EC1FF205E
:1051000009F49FC1EE2009F44FC1802F0E943B2675
:10511000093309F08FC1FFEF21EE84E0F150204008
:105120008040E1F700C00000E4C1E1108CC1812F94
:105130000EC1812F837009F070C0F110DAC1202FE9
:10514000229526952770220F220F602F6F70862FD1
:1051500090E0A0E0B0E06C017D01022E04C0CC0C18
:10516000DD1CEE1CFF1C0A94D2F704FF12C08FE076
:1051700090E0A0E0B0E004C0880F991FAA1FBB1FF9
:105180002A95D2F7BC01CD016095709580959095D8
:1051900003C060E070E0CB011695169513701230D5
:1051A000B1F040F56C297D298E299F29113031F10C
:1051B0000F900F900F900F900F90DF91CF911F9154
:1051C0000F91FF90EF90DF90CF900C94E12E6C291F
:1051D0007D298E299F290F900F900F900F900F908F
:1051E000DF91CF911F910F91FF90EF90DF90CF90C3
:1051F0000C94FB2E0E94E12EC701B6010F900F9078
:105200000F900F900F90DF91CF911F910F91FF9012
:10521000EF90DF90CF900C94C72EFF2019F0812FD4
:10522000817001C08695882309F463C1202F2295DF
:1052300026952770220F220F602F6F70862F90E027
:10524000A0E0B0E06C017D01022E04C0CC0CDD1C9E
:10525000EE1CFF1C0A94D2F704FF12C08FE090E00E
:10526000A0E0B0E004C0880F991FAA1FBB1F2A95B9
:10527000D2F7BC01CD01609570958095909503C0E3
:1052800060E070E0CB011695169513701230B1F006
:1052900040F56C297D298E299F29113031F10F901D
:1052A0000F900F900F900F90DF91CF911F910F9162
:1052B000FF90EF90DF90CF900C94A82F6C297D2960
:1052C0008E299F290F900F900F900F900F90DF91D4
:1052D000CF911F910F91FF90EF90DF90CF900C94A2
:1052E000BA2F0E94A82FC701B6010F900F900F9000
:1052F0000F900F90DF91CF911F910F91FF90EF9042
:10530000DF90CF900C94962F023F09F45EC008F412
:1053100049C0033F09F46CC0F2CE902F9071E92E82
:10532000812F8F71FF2051F00E942F2F802FEE20B0
:1053300019F08295807FBECE8F70BCCE0E94502F18
:10534000802FEE2019F08295807F01C08F700F9022
:105350000F900F900F900F90DF91CF911F910F91B1
:10536000FF90EF90DF90CF900C948927FF20A9F059
:10537000E4E0EE1508F4BDC0812F8F710F900F90FF
:105380000F900F900F90DF91CF911F910F91FF9091
:10539000EF90DF90CF900C94752FF5E0FE1508F498
:1053A000A8C0EACFFF2099F0812F8F710F900F9046
:1053B0000F900F900F90DF91CF911F910F91FF9061
:1053C000EF90DF90CF900C942F2FFF2069F3812F67
:1053D0008F710F900F900F900F900F90DF91CF91E2
:1053E0001F910F91FF90EF90DF90CF900C94502F72
:1053F000FF2089F0812F8F710F900F900F900F90E9
:105400000F90DF91CF911F910F91FF90EF90DF9060
:10541000CF900C941A2F0F900F900F900F900F9029
:10542000DF91CF911F910F91FF90EF90DF90CF9080
:105430000C94152F033509F46ECE073409F059C0CA
:105440006ACEEE2021F2802F0F900F900F900F90D8
:105450000F90DF91CF911F910F91FF90EF90DF9010
:10546000CF900C942B27412F4F70602FC6010E94C4
:1054700094310F900F900F900F900F90DF91CF917C
:105480001F910F91FF90EF90DF90CF900C94212E01
:1054900001112FC0FF2069F10E9496272FEF80E7AE
:1054A00092E0215080409040E1F700C000000F9052
:1054B0000F900F900F900F90DF91CF911F910F9150
:1054C000FF90EF90DF90CF900C947531412F4F708B
:1054D000602FC6010F900F900F900F900F90DF91EB
:1054E000CF911F910F91FF90EF90DF90CF900C9490
:1054F00097310F900F900F900F900F90DF91CF91F9
:105500001F910F91FF90EF90DF90CF9008951F9320
:10551000CF93DF9300D000D01F92CDB7DEB7942F8A
:105520004983252F5A836B837C838D834C815D81D6
:10553000452B31F02F3F31F481E09F3F19F403C038
:1055400081E001C080E0182F117080FD31C04981D9
:105550005A816B817C818D810E94CD2F292F2295CC
:105560002F702C3030F42A30A0F42250223030F04A
:1055700022C02C30C9F02F30B9F01DC0853A28F474
:105580008430C0F4823028F415C090E2980F98302F
:1055900088F0883E30F4803E68F48450813A58F4B4
:1055A00009C0803F41F406C093FB112710F903C0E6
:1055B00010E001C011E0812F0F900F900F900F901D
:1055C0000F90DF91CF911F910895CF93DF9300D07B
:1055D00000D01F92CDB7DEB70F900F900F900F90B5
:1055E0000F90DF91CF910895CF93DF9300D000D03B
:1055F00000D0CDB7DEB726960FB6F894DEBF0FBE4B
:10560000CDBFDF91CF9108951F93CF93DF93C091CA
:105610005B0416E080915C04C81799F0D0E01C9FF1
:10562000F0011D9FF00D1124E35AFB4F4081518181
:1056300062817381848195810E94F42A2196C770CA
:10564000E9CFDF91CF911F91089540918D04509142
:105650008E0460918F0470919004809191049091D8
:1056600092040C94F42A0F931F93CF93DF938091AD
:10567000920482958F7009F05DC080918F04882319
:1056800009F458C080915B0410915C0460918D0412
:1056900070918E04C0919004D091910491E06F3F7D
:1056A00009F090E0292F06E0811709F443C0209704
:1056B00021F07F3F21F030E003C031E001C0322F04
:1056C00090E030FD34C0089FF001099FF00D1124D7
:1056D000DF01A35ABB4F11963C911197371327C096
:1056E0003C91361324C012963C91129731111FC081
:1056F00013964D915C9114974C1B5D0B483C5105E2
:10570000B0F4809192048F70806180939204EE597E
:10571000FB4F80818F70806180838DE894E00E94D0
:105720009A27DF91CF911F910F910C94042B019632
:105730008770BACFDF91CF911F910F9108959F92FB
:10574000AF92BF92CF92DF92EF92FF920F931F938F
:10575000CF93DF93CDB7DEB761970FB6F894DEBF76
:105760000FBECDBF8C0185E0F801DE011D960190D2
:105770000D928A95E1F7F80140815181F280C38052
:10578000D48090918D0460918E042091900430918A
:1057900091042115310531F06F3F31F481E09F3FD5
:1057A00019F403C081E001C080E0F82FF1709F2E52
:1057B00080FD52C18DE8A82E84E0B82EE0908F04C1
:1057C000F601E21BF30BEE2009F4E8C0809192048D
:1057D000E83CF10508F0A4C0282F207F09F053C051
:1057E000561313C0491311C0EF2CF1100EC08F7067
:1057F0008061809392040E94252BC5010E949A2704
:1058000080919204F80185835BC1C114D10431F009
:105810005F3F31F481E04F3F19F403C081E001C0E4
:1058200080E080FD03C081E08F2502C080E090E031
:10583000F82FF170EF2E80FF1CC080915B04209147
:105840005C0436E0821709F418C190E0389FF0013B
:10585000399FF00D1124E35AFB4F6181561306C0A6
:105860006081461303C06281F61203C001968770FF
:10587000E9CFEF2CFF2009F423C1809192048160CD
:105880008093920462C0561306C0491304C0F110FD
:1058900002C0F801A7C04D875E87FF867C2DD98A9C
:1058A000C88A6F2D89890E94872A882399F1FF2051
:1058B00089F120919204822F82958F7090E0029757
:1058C00074F080918D0490918E0498878F8319864F
:1058D000DB86CA862C87CE0107960E949A2786E02F
:1058E000F801ADE8B4E001900D928A95E1F70E94CD
:1058F000332B0E94252B11C0561749F14D875E8727
:10590000FF867C2DD98AC88A6F2D89890E94872AB3
:1059100081112CC0C8010E949A27EE24E394D0C0C4
:10592000282F207F49F77C2DD98AC88A6F2D898935
:105930000E94E52A8DE894E00E949A2786E0F5010E
:1059400011928A95E9F70E94252BE12CB9C04913E1
:10595000D5CFF110D3CFF8018583C8010E949A27D3
:1059600086E0F50111928A95E9F7AAC0FF2091F22D
:1059700020919204822F82958F7090E002970CF410
:10598000AECF80918D0490918E049A8389831B827F
:10599000DD82CC822E83CE0101969FCFE83CF105BB
:1059A00008F04BC0EF2CFF2009F4B4CF561330C0E1
:1059B00049132EC02091920420FD21C0822F829590
:1059C0008F70482F50E041155105C9F0F80125832B
:1059D0004F30510541F08F5F982F9295907F822F25
:1059E0008F70892B8583C8010E949A2786E0F80171
:1059F000ADE8B4E001900D928A95E1F72AC086E007
:105A0000F801ADE8B4E001900D928A95E1F758C035
:105A10004D875E87FF867C2DD98AC88A6F2D89893C
:105A20000E94872A81115BCF8091920481608093CC
:105A30009204C8010E949A2743C07C2DD98AC88A43
:105A40006F2D89890E94E52A86E0F50111928A95D9
:105A5000E9F70E94252B34C0FF2009F45BCF4D8766
:105A60005E87FF867C2DD98AC88A6F2D89890E941E
:105A7000872A882309F44ECF32CF7C2DD98AC88A51
:105A80006F2D89890E94CD2F292F22952F702230CA
:105A900028F49F7039F0811105C00BC0243028F420
:105AA0009F7049F4805E883020F0C8010E949A27D8
:105AB0009E2CE92C05C0F8019581907F99F7F9CFCC
:105AC0008E2D61960FB6F894DEBF0FBECDBFDF916D
:105AD000CF911F910F91FF90EF90DF90CF90BF90EB
:105AE000AF909F9008951F93CF93DF93CDB7DEB70C
:105AF0002C970FB6F894DEBF0FBECDBF4F835887EB
:105B000069877A878B879C87CE0107960E949F2B97
:105B10008823D1F09F8188852A853B85232B31F00E
:105B20008F3F31F481E09F3F19F403C081E001C051
:105B300080E080FD47C04F81588569857A858B85D7
:105B40009C850E94F42A3EC086E0FE013796DE0165
:105B5000119601900D928A95E1F7FF81E8856A859B
:105B60007B856115710531F0EF3F31F481E0FF3F36
:105B700019F403C081E001C080E080FD23C02091C2
:105B80005C0430E0C90101968770992740915B045D
:105B900050E084179507F1F1F983EA837D836C83E4
:105BA00096E0929FD001939FB00D1124A35ABB4F52
:105BB000FE01319601900D929A95E1F780935C0475
:105BC0000E94042B16E080915B0490915C0489177D
:105BD00071F1189FC0011124835A9B4F0E949F2B83
:105BE000882329F1E0915B041E9FF0011124E35A00
:105BF000FB4F4081518162817381848195810E9434
:105C0000F42A80915B0490E0019687709927809335
:105C10005B04D9CF0E94962710925C0410925B041B
:105C2000EDE8F4E086E0DF011D928A95E9F72C9615
:105C30000FB6F894DEBF0FBECDBFDF91CF911F919D
:105C40000895DF92EF92FF920F931F93CF93DF930C
:105C5000FC01892B09F488C0E12CF12CDD24D394BC
:105C6000EF0121968491853709F460C058F4843798
:105C700008F04EC0843008F068C08130D1F0823026
:105C800071F172C0883709F45BC050F4863709F4AB
:105C900053C0873709F068C08E2D0E949C3052C0D7
:105CA0009CE7980F903708F05FC08F770E942B27F2
:105CB0004EC08F010E5F1F4FFE01849190E2980F3E
:105CC000983050F48770FD2D01C0FF0F8A95EAF7D8
:105CD0008F2F0E94A23015C00E943B2614C08F0156
:105CE0000E5F1F4FFE01849190E2980F983068F488
:105CF0008770FD2D01C0FF0F8A95EAF78F2F0E9454
:105D0000A8300E94C930E80122C00E942B27FBCF97
:105D1000CF010296FE01C491CC2361F0EFE9FFE0D0
:105D20003197F1F700C00000C150F6CFCF010296C5
:105D3000FE01F490EC010BC00E948C30E82E07C0ED
:105D40000E949F300E94C93002C00E943B268F2DC6
:105D5000882341F0EFE9FFE03197F1F700C0000040
:105D60008150F6CFFE017CCFDF91CF911F910F9133
:105D7000FF90EF90DF9008956093930570939405E2
:105D800080939505909396050C94053108950F9393
:105D90001F930091970510919805209199053091D6
:105DA0009A05602B712B822B932B60939705709330
:105DB00098058093990590939A051F910F910C94E3
:105DC00004310F931F93009197051091980520912E
:105DD000990530919A056023712382239323609360
:105DE0009705709398058093990590939A051F9154
:105DF0000F910C9404310F931F930091970510910C
:105E000098052091990530919A056027712782277E
:105E100093276093970570939805809399059093C5
:105E20009A051F910F910C94043160E070E0CB0152
:105E30000C94BC2E0F931F9341E050E060E070E0A3
:105E40008A019B0104C0000F111F221F331F8A9576
:105E5000D2F7C901B8011F910F910C94BC2E0F937A
:105E60001F9341E050E060E070E004C0440F551F14
:105E7000661F771F8A95D2F78091930590919405BC
:105E8000A0919505B09196058A019B01082B192BCD
:105E90002A2B3B2BC901B8011F910F910C94BC2EEA
:105EA0000F931F9341E050E060E070E004C0440FA6
:105EB000551F661F771F8A95D2F7409550956095BC
:105EC00070958091930590919405A0919505B0915E
:105ED00096058A019B01082319232A233B23C90124
:105EE000B8011F910F910C94BC2E0F931F9341E0AA
:105EF00050E060E070E004C0440F551F661F771F3C
:105F00008A95D2F78091930590919405A09195057B
:105F1000B09196058A019B01082719272A273B275C
:105F2000C901B8011F910F910C94BC2E0F931F93C0
:105F30000091930510919405209195053091960557
:105F4000602B712B822B932B1F910F910C94BC2EE5
:105F50000F931F930091930510919405209195053F
:105F60003091960560237123822393231F910F9113
:105F70000C94BC2E0F931F930091930510919405E0
:105F800020919505309196056027712782279327E8
:105F90001F910F910C94BC2E08958F929F92AF92F7
:105FA000BF92DF92EF92FF920F931F93CF93DF93F5
:105FB00000D000D01F92CDB7DEB76B837C838D837A
:105FC0008A018C819D81892B31F01F3F31F481E062
:105FD0004F3F19F403C081E001C080E080FF03C09F
:105FE00080E090E04DC08B818823D1F180909305B3
:105FF00090909405A0909505B09096058091970596
:1060000090919805A0919905B0919A05882A992AAE
:10601000AA2ABB2A8FE1E82EF12CD501C4010E2C4F
:1060200004C0B695A795979587950A94D2F780FDF9
:1060300006C081E0E81AF10880F7D12C07C0DE2CF9
:10604000B8018E2D0E94B331019799F380E1189F1A
:10605000F0011124ED56FB4FE00FF11DD08209C075
:1060600080E1189FF0011124ED56FB4FE00FF11D68
:10607000D08009831A8369817A818D2D0E94B33182
:106080000F900F900F900F900F90DF91CF911F9175
:106090000F91FF90EF90DF90BF90AF909F908F9007
:1060A00008952091130130911401F90132969FEF68
:1060B00040E05191851789F09F3F19F4511101C0BB
:1060C000942F4F5F4630A9F79F3F39F0F901E90F50
:1060D000F11D97FDFA95828308950895E0911301CB
:1060E000F09114019F012A5F3F4F9281891301C0F3
:1060F00012823196E217F307C1F7089581E090E02C
:10610000E0911301F0911401E80FF91F108201963C
:1061100088309105A9F708958091A505089590917B
:10612000A505892B8093A505089580959091A505D7
:1061300089238093A50508958093A505089510925D
:10614000A50508959091A405892B8093A405089531
:1061500080959091A40589238093A40508951092B9
:10616000A405089580939B05089510929B050895BA
:106170008091130190911401FC0131969C01285FDC
:106180003F4F80E0919191118F5FE217F307D1F7B4
:106190000895E0911301F09114018091A505808389
:1061A000E0911301F091140190818091A405892B55
:1061B000808380919B05882361F0E0911301F09129
:1061C00014019081892B80830E94B8308111109234
:1061D0009B0580911301909114010C948F2490934E
:1061E00087018093860108950895CF93DF9300D0AF
:1061F00000D01F92CDB7DEB70F900F900F900F9089
:106200000F90DF91CF910895089508950C94EF2594
:1062100080E008958091AC05843021F11092A705AB
:1062200020E488E190E00FB6F894A8958093600090
:106230000FBE2093600083B7817F846083BF83B7E4
:10624000816083BF7894889583B78E7F83BF0FB6B4
:10625000F894A89580916000886180936000109206
:1062600060000FBE0895CF930E94F3250E94280678
:106270000E94F425C0E08C2F0E941007892B29F47E
:10628000CF5FC031C1F780E001C081E0CF910895B8
:106290000E94F1250C9496271F920F920FB60F9231
:1062A00011248F939F93AF93BF938091A705811182
:1062B00013C080911C0390911D03A0911E03B09107
:1062C0001F034196A11DB11D80931C0390931D03D4
:1062D000A0931E03B0931F03BF91AF919F918F9125
:1062E0000F900FBE0F901F9018950E941A23F894DC
:1062F00087E797E7909301088093000887E090EB89
:10630000DC018093B5059093B605A093B705B093D3
:10631000B8059CE088E10FB6F894A89580936000DA
:106320000FBE90936000FFCF80E090E00895089545
:10633000E72FF0E090E1899FE00DF11D112484E04A
:10634000EE0FFF1F8A95E1F7E60FF11DE052FF4FB8
:1063500084910895E82FF0E0EE0FFF1FE05AF0401F
:106360008591949108950E94983190E4980F90320D
:1063700018F40E94AA3108958F3B50F4883A48F5EA
:10638000853AD0F48430A8F4813009F4B2C0AEC0AC
:10639000883E40F4803E68F48F3B09F0A7C020E0BF
:1063A00030EEA9C0803F08F4A1C0282F30E030654E
:1063B000A2C0282F30E09FC0853A29F0863A31F0FC
:1063C00023E830E498C021E830E495C022E830E4C6
:1063D00092C0883A09F445C0893A09F445C08A3A1E
:1063E00009F445C08B3A09F445C08C3A09F445C01C
:1063F0008D3A09F445C08E3A09F445C08F3A09F444
:1064000045C0813B09F445C0803B09F445C0823B4F
:1064100009F445C0833B09F445C0843B09F445C0F9
:10642000853B09F445C0863B09F445C0873B09F428
:1064300045C0883B09F445C0893B09F445C08A3B07
:1064400009F445C08B3B09F445C08C3B09F445C0B9
:106450008D3B09F445C08E3B09F445C020E034E48F
:106460004AC022EE34E447C029EE34E444C02AEEA8
:1064700034E441C025EB34E43EC026EB34E43BC0B9
:1064800023EB34E438C024EB34E435C027EB34E4A8
:1064900032C02CEC34E42FC02DEC34E42CC023E8C3
:1064A00035E429C02AE835E426C022E935E423C0D2
:1064B00024E935E420C021E236E41DC023E236E4BD
:1064C0001AC024E236E417C025E236E414C026E2FE
:1064D00036E411C027E236E40EC02AE236E40BC0EF
:1064E0002FE634E408C020E734E405C020E030E0C3
:1064F00002C021E030E0C90108950E94EE3208F4A4
:1065000081E008950E94423388F09F5798F0B92F98
:106510009927B751B0F0E1F0660F771F881F991FD8
:106520001AF0BA95C9F714C0B13091F00E945C33EB
:10653000B1E008950C945C33672F782F8827B85FFB
:1065400039F0B93FCCF3869577956795B395D9F730
:106550003EF490958095709561957F4F8F4F9F4F3A
:106560000895E89409C097FB3EF490958095709546
:1065700061957F4F8F4F9F4F9923A9F0F92F96E98F
:10658000BB279395F695879577956795B795F11104
:10659000F8CFFAF4BB0F11F460FF1BC06F5F7F4FA1
:1065A0008F4F9F4F16C0882311F096E911C07723B3
:1065B00021F09EE8872F762F05C0662371F096E8BC
:1065C000862F70E060E02AF09A95660F771F881F8B
:1065D000DAF7880F9695879597F90895990F00082F
:1065E000550FAA0BE0E8FEEF16161706E807F907A5
:1065F000C0F012161306E407F50798F0621B730B40
:10660000840B950B39F40A2661F0232B242B252BC0
:1066100021F408950A2609F4A140A6958FEF811D63
:10662000811D089597F99F6780E870E060E0089504
:106630009FEF80EC089500240A941616170618069A
:106640000906089500240A94121613061406050676
:106650000895092E0394000C11F4882352F0BB0F07
:1066600040F4BF2B11F460FF04C06F5F7F4F8F4F6A
:106670009F4F089557FD9058440F551F59F05F3FA5
:1066800071F04795880F97FB991F61F09F3F79F054
:1066900087950895121613061406551FF2CF4695D6
:1066A000F1DF08C0161617061806991FF1CF869558
:1066B0007105610508940895E894BB27662777273C
:1066C000CB0197F908950E94EE3208F48FEF0895F8
:1066D0000E947B330C9429330E941B3338F00E94B4
:1066E000223320F0952311F00C9412330C941833BC
:1066F00011240C945D330E943A3370F3959FC1F3DB
:10670000950F50E0551F629FF001729FBB27F00D5F
:10671000B11D639FAA27F00DB11DAA1F649F6627B4
:10672000B00DA11D661F829F2227B00DA11D621F03
:10673000739FB00DA11D621F839FA00D611D221FBD
:10674000749F3327A00D611D231F849F600D211DA1
:10675000822F762F6A2F11249F5750409AF0F1F024
:1067600088234AF0EE0FFF1FBB1F661F771F881F8D
:1067700091505040A9F79E3F510580F00C94123380
:106780000C945D335F3FE4F3983ED4F386957795A0
:106790006795B795F795E7959F5FC1F7FE2B880F33
:1067A000911D9695879597F90895EE0FFF1F059017
:0A67B000F491E02D0994F894FFCF56
:1067BA008000052A030000FFD51CDA1CD81C131E12
:1067CA00D91C019C0566756C6C006C6F7700000023
:1067DA000000E50400000000E40400000000CD0809
:1067EA0021047104470B8C04230424048F049404A9
:1067FA00990465046E04A104FEFF0000DA04000097
:10680A000000C50C00000000350D3B0D310D340DA4
:10681A002B0D2E0D2E0D00000000560EFD0DB60E8E
:10682A0000000000011921046018081C5818641A95
:06683A0024045B18260493
:00000001FF
